:020000041100E9
:103000007FB50023284C294D03932800217C284AB2
:1030100001F0E1FA002812D103232800217C03AA41
:1030200001F080FA00280AD1224B039A9A4206D175
:10303000214B2248E360224B636104B070BD02263D
:10304000217CFE2228001F4B009601F03DFA00284B
:1030500001D00020F1E71C4BA2899A42F9D1217CD2
:10306000FF222800194B009601F02EFA0028F0D11B
:10307000E389174A934203D1164B17486361DCE793
:10308000164A9342E5D1164B164A1B68934206D95D
:10309000C02304222800217C9B0001F07EFA124B01
:1030A00012486361C9E7C0460062FF1F3442FF1F38
:1030B000813700005959530059598320D0BE00115F
:1030C000094200110C62FF1F595900000E62FF1FD8
:1030D00083050000BD410011B0BE00118215000043
:1030E0002462FF1F87130000C5420011C0BE0011FB
:1030F000002370B51A4E1B4C30006361637401F0FD
:1031000091F9402323744B2B0CD9CC233821AC22CA
:1031100030009B01217401F040FA00280AD00025FC
:1031200025740CE0FFF76CFF051E08D1237C0433E7
:10313000DBB2E7E70C4B0D4D63610D4BE381236878
:10314000002B08D1002D06D00C222900200008F009
:1031500083FD2B7B6374300001F0A2F970BDC04683
:103160003442FF1F0062FF1F5D420011A0BE00112C
:10317000AAAAFFFFF7B5164B0192C318021D002043
:10318000009388235B05D3181B685C1C1AD09CB283
:10319000402C18D88D781E0CAC466746CD782D0291
:1031A0003D43AE4206D1019800280ED110000C70AC
:1031B000240A4C7003249BB20733A343D218009B0C
:1031C0009A42DED3FEBD4432F9E71000FAE7C0466A
:1031D000FC0F0000802213B503000324019189B283
:1031E000520107319B18A14304305A1A88235B050A
:1031F000C3181B68591C03D190429241104016BD60
:1032000099B2402907D80B000733A343C018904256
:10321000ECD30020F3E74430F9E7134B134A1B6863
:10322000126810B5FA24934201D81A00F824104B02
:10323000E4021B689A4210D813000E4A12689A42A0
:103240000ED3013307D1F823DB029C4203D10A4994
:10325000054808F0B1FB200010BDFC24E402ECE7B7
:10326000FE24E402F7E7C04600C0071100D00711B2
:1032700000E0071100F00711FFFFFF7FF0B59BB0E2
:10328000150004900391402A00D9A0E006AB5980B4
:103290001A80FFF7C2FF0400042816D9002206A9ED
:1032A000FFF768FF052810D906AB1B88AB420CD18D
:1032B000002D07D0514B2A000499C01808F0A4FC37
:1032C000002802D101201BB0F0BD06AB1D802000FC
:1032D0000699FFF77FFF041E7BD1069B0793FFF73C
:1032E0009CFF80235B01C618802307001B039E42BE
:1032F00001D3F826F60288235B05F31801931B68B7
:10330000013302D0019808F007FB3D49019808F00D
:1033100053FB3B1D0293331D05938822029B5205EC
:103320009B181B6808935A1C3CD044219AB2009108
:10333000402A04D80320D11D814389B2009103990A
:103340001B0C8B4224D0402A22D80122300008A92D
:10335000FFF710FF021E1BD1380008A9FFF70AFF74
:103360000400042831D9009A059B9B188022520141
:10337000B218934240D288235B05C118009A09A86D
:1033800008F06AFC1D4B009A09A9F01808F0CCFC63
:10339000009A029B9446634402931A4B029AFB18CC
:1033A0009A42BAD388235B05FC1821680198013939
:1033B00008F002FB200008F0AFFA039A07AB5A802E
:1033C00030000799FFF706FF0400002C03D100200E
:1033D00079E70428FBD988235B05E018069908F0F3
:1033E000EBFA0323EA1C9A4300D16BE7034B0499E1
:1033F000E01808F099FC65E70424ECE704000011EC
:10340000FFFFFF7FF80F0000F7B505001400402A0A
:1034100021D8002701AE71803780FFF7FEFE042817
:1034200016D93A003100FFF7A5FE042810D93688D6
:10343000BC420BD0BD4209D0221CB44200D9321C80
:10344000064B92B2C118280008F006FC30B2FEBD4F
:10345000C04300B2FBE703204042F8E7040000113C
:1034600037B5042204000D0001A81649FFF7CCFF70
:10347000020004280BD1019BA34208D3AB4204D025
:10348000104901A80195FFF7F9FE01203EBD0E4C41
:1034900023682000019308F03FFA019920000139C8
:1034A000019108F089FA80235B01E418074B9C42E4
:1034B000EED10422034901A80195FFF7DFFE0020A9
:1034C000E4E7C0465555000000C007110000081190
:1034D00030B589B008F0F8FB10226946254808F09D
:1034E00093F9254B009A9A420ED1019B029A0F2B19
:1034F00033D8002101240698013B08D2002900D0CE
:103500000292029B013331D10023029325E0551C26
:10351000F2D102002100EFE710341022200004A9AC
:1035200008F072F9029B013301D1069B02938823B4
:1035300004995B05C918059B06981A03120B0491A0
:103540000592814203D02B4201D108F085FB019BFB
:10355000013B0193019B002BDED1029B002B03D08A
:10356000049304984168084709B030BDE025014C38
:103570002D03EFE700000111504859368022F8B5BD
:10358000964C974BD200002120001C6008F0C4FB31
:103590002300944A88331A60934B1A786A23002ACE
:1035A00000D01133E3620A232365904B37221B7846
:1035B0000820A3638E4B2118E361102323628D4BF7
:1035C0003B256361C823DB00A36123008C331A60B1
:1035D0002823013AE26320646364CA67043A211D28
:1035E000CA672100BC310D602100C0310860210094
:1035F000C4310B6021000635CC310D602100083D3F
:10360000C8310D602100D0310A602200D432106030
:103610002200D832136022000227E0322100176016
:103620004222DC310A6021001B3DE4310D602100A3
:10363000E83108602100EC310B6023000521F433F0
:1036400019602300F0331A602300183290331A6097
:1036500023009433186023001E3A98331A60AF2376
:10366000DB002360644BFA262363644B644DE36004
:10367000644BF031A3642300FF31FC33B600A1603A
:1036800021611E60A5627325E5656D3D6565A565D3
:1036900096255D4AAD00E264666258606766A5667D
:1036A00000270925A767E566584F594D6067200038
:1036B0002567E2673A6015279C30676007001A208B
:1036C00038602000A0300700212038602000A8309A
:1036D00007004C4838602000F83006602600642758
:1036E000A436376026005F3FAC3637602600033FC4
:1036F000B03637602600C637B4363760260000275C
:10370000B836376038269E60424E96205E64424E40
:103710005A66DE61414E9A645E62F53EFF3E9E62ED
:103720001E269A67354A8000DE661F675F67DD6583
:103730001D661862DA67BE23394A5B00E250394BD6
:10374000D838235004302250C4225200A350C6233C
:10375000E4205B00E1500433334AE1503349344BF9
:10376000D1603449800019503349E938FF38195085
:1037700032490430195032493248D161324911631B
:10378000324951631900F4310860CE2030494000BD
:1037900011603049195019002F48F83108602F493D
:1037A000D16582212E4A89005A501A002D490832CB
:1037B000D1671A002C49B432116088212B4A890044
:1037C0005A501A002A49883211602A4ADA6408F0ED
:1037D0006BFA012008F030FAF8BDC0460004FF1F64
:1037E000A464FF1F706FFF1F7044FF1F4A0AFF1F72
:1037F0003A07000080C3C9019A020000DC050000FE
:103800006A18000050C3000088130000F009FF1F71
:10381000204E00006509FF1F68100000C409000069
:1038200040420F0010270000FC00FF1FB11CFF1FCB
:103830000000FF1F052DFF1F8D30FF1F252FFF1FCD
:103840007120FF1F6127FF1F8D20FF1F3922FF1FDF
:10385000FD1FFF1F8529FF1F6D2AFF1F8D19FF1FE9
:103860009128FF1FB525FF1FC125FF1FFD1EFF1F4C
:10387000B51FFF1F751EFF1F0223F0B50124624D07
:10388000624E2B70624B91B01C70624F0393336891
:1038900000210820FB7006F061FE082006F058FDAC
:1038A0000023984205D0FA78552A02D0332A00D056
:1038B0009DE03360042006F0CBFF08F08DF8FFF7A1
:1038C0005DFE08F0B1F81F2201240021524B10AE1A
:1038D0001A70524B1C70524B1970524B196891431D
:1038E000163A0A431A60602219689143403A0A4323
:1038F0001A6007F0F1FF08F02FF94B4B9847C120F1
:10390000FF214A4B80001A588A431A50C522920060
:1039100098588843BF390143995098584449084002
:103920008021C9010143802099509958C00509029E
:10393000090A0143995080213E48490107F024FFBC
:10394000032322003C49019400933C4807F0BCFF4C
:103950002C223B4905A808F07FF905AC6178207856
:10396000023406F015FDA642F8D1364C00200121A4
:1039700006F022FE2268344B03201A40A023DB020B
:1039800013432360802322689B041343236022682F
:103990002E4B1A4080239B03134323602C4A2D4B4C
:1039A000934200D8012008F0C7F808F05DF98023A1
:1039B0002268DB0413432360287807F045FF039B4C
:1039C0001878C0B207F0F0FE08F0CEF822490420C3
:1039D00008F0AAF806F008FF00F040F800F030FE0A
:1039E00000F0D8FE00F018FA002011B0F0BD0093EE
:1039F0002100194A042008F0CFF88023DB059C62DF
:103A0000FFF766FD56E7C0464A0AFF1F34F0004044
:103A10007044FF1F3062FF1F480AFF1F490AFF1F43
:103A2000680AFF1FBCF00040E1A2000000E100E0D6
:103A3000FF00FFFF7444FF1FF856FF1F7454FF1F61
:103A4000C8BD001114F00040FF7FF8FFFFFF9FFF8B
:103A50000080FF1F706FFF1F3B000108002210B5A0
:103A60001100112007F080FF10BD0000F8B5002301
:103A70000926374F374C3B62E3681120B343E360BC
:103A800008F072F9112008F007F9112008F034F855
:103A90004023226880251343236080236268DB0271
:103AA00013436360A3682C4A2B43A360A3680221DD
:103AB0001340A3608023A2689B0113431022A360DC
:103AC000236C072093432364236C0F3A134323642E
:103AD00080235B003B62226B204B1A402263626BA7
:103AE0001A406263A26B1A40A263E26B1340E36365
:103AF000E3681B4A1340E36006F04AFC01210720FB
:103B000006F05AFD174B11205A6C15435D6407F0FF
:103B100073FEFD21144B154A89005A508023C7209B
:103B2000626B5B0313436363E36880003343E360CA
:103B30000F4B104A19581140802212020A431A50A2
:103B4000802292051A6008220B4B5A63F8BDC046CA
:103B500000F000403CF00040FFFFDFFFEFFFEFFF11
:103B6000FFFF7FFF003800400000FF1F5118FF1FBC
:103B700000E100E0FF00FFFF00000540E12010B57C
:103B8000C00407F0E1FE10BD70B52B4C238C002B58
:103B90002AD0FA22D200934201D2FFF7EFFF228A05
:103BA000238C002A21D1DA0023826382A382E3825C
:103BB00023836383A383E38322606260A260E26065
:103BC0001E4D1F4A6420EB8093420AD8FA2200203F
:103BD000D200934205D91B4A0A21981807F024FE07
:103BE000C0B200232872238470BD0720E11CCA7F65
:103BF00001320240CA7705D10325201DC17F013162
:103C00002940C17708325200A352002321001A0034
:103C1000088A01321B180231082AF9D1221DD27FED
:103C20009200A350626823689B18A2689B18E26800
:103C30009B185B099BB2C3E77061FF1F1862FF1FEF
:103C4000B70B000030F8FFFF30B503A804880B2045
:103C5000002C0ED14968074D0878497809020143C4
:103C60000A20A94205D1012120001980024B1B7AAC
:103C7000137030BD192A00001862FF1FF7B5150038
:103C800008AA16884A680F4F147852781202224305
:103C90000A24BA4214D10122DBB2019200962A0012
:103CA00007F0F2FC041E0BD1074B1B68002B07D05A
:103CB00068782A7800021043424250410130984708
:103CC0002000FEBD022900009C61FF1F30B50125C8
:103CD00003790400BFB02B4211D00A49408807F095
:103CE0003FF828420BD0084B01A95B8D4D800B801B
:103CF000064B00221B7A60880B7104F011F93FB06B
:103D000030BDC0469461FF1FA840FF1F1862FF1F0F
:103D100010B50549054806F0D9FF0421044A0548B5
:103D200006F096FF10BDC0469461FF1FFFFF000024
:103D3000F4BD0011A840FF1F10B5024804F072FF47
:103D400010BDC046CD3C0011012303700B4B1A7A05
:103D50004270022282709A78C270DA78027103226D
:103D600042711A7982715A79C2710C2202729A795F
:103D70004272DB7983720B207047C0461862FF1FC6
:103D8000022310B50370013B437005338370103379
:103D90000371443B43712A3383714433C37100235D
:103DA0000372064B04001B8843720A30FFF7CCFFF6
:103DB000831D0A30C0B2E37010BDC0461862FF1FF9
:103DC00010B5142007F090FF124B14220021186048
:103DD00007F0A2FF002007F087FD012007F074FE26
:103DE000022007F0E1FE032004F0C0F9042006F0F1
:103DF000D5F9052003F0FEFB062004F0CBF80720E0
:103E000001F0B4FA082006F003FF092001F080F861
:103E100010BDC046A061FF1F07F01EFE012007F085
:103E2000FBFE07F099FD0000094B10B50400984215
:103E300005D0012904D12000064906F047FF10BD36
:103E40000229FCD1013904F0ABFE0028F3D0F6E7DB
:103E5000FEFF0000C661FF1F70B50D7A100004AAB6
:103E60002C00168810221440154220D1002E20D19B
:103E70000A78022A18D14A68517815780E4A090240
:103E80002943914205D00D4A914209D01C800A2451
:103E900004E014220A491A8007F0DEFE200070BDFB
:103EA0000C2208491A80F7E71C800124F6E7082451
:103EB000F4E70B24F2E7C046F3FF0000F4FF000034
:103EC000FC42FF1FECBE001110B504000749084872
:103ED00006F0FCFE074804F0E5FD0020E40704D5E9
:103EE0000721054A054806F0B3FE10BDC661FF1F55
:103EF000FFFF0000293E001138BE0011EC40FF1FFB
:103F000000B50C4BBFB01A780B4902A800F0FCFCBE
:103F10006B4680B2D880002809D06A46074B01A9B9
:103F20001B889380064B0022188803F0F9FF3FB0EE
:103F300000BDC046A461FF1FA561FF1F4641FF1FD2
:103F40005042FF1F00B50C4BBFB01A780B4902A8B6
:103F500001F02CFF6B4680B2D880002809D06A4659
:103F6000074B01A95B8D9380064B0022188803F054
:103F7000D7FF3FB000BDC046CE61FF1FCF61FF1F1E
:103F8000EC40FF1F5042FF1FF7B50E00377A1C00B0
:103F900008AB11003D001A8820231D401F423CD170
:103FA0003378022B3BD173681F785B781B023B434D
:103FB0001E4FBB4208D01E4FBB4214D01D4DAB421A
:103FC00021D00A252800FEBD002A2AD1142C2AD887
:103FD0002200F06807F040FE174B1C70012CF1D94D
:103FE000FFF7B0FFEEE7002A1BD1202C1BD82200E0
:103FF000F06807F031FE114B04211C70104B18784B
:1040000007F06AFEDEE7E3B20124009201940A00A1
:10401000310007F039FB0500D4E70825D2E7012578
:10402000D0E70B25CEE70D25CCE7C046F3FF000017
:10403000F4FF000002290000CE61FF1FA461FF1FF2
:104040005062FF1F332310B5040003700A22074992
:10405000013007F001FE064B0F201B681A0AE372BD
:1040600022731A0C1B0E6273A37310BD1862FF1F1C
:104070004062FF1F30B5012503790400BFB02B4219
:1040800013D00B49408806F06BFE28420DD06A46DB
:10409000084B02A81B889380FFF7D4FF6B46D8809B
:1040A0000022608801A903F03BFF3FB030BDC0464D
:1040B000C661FF1F4641FF1F10B5024804F0B2FD64
:1040C00010BDC0467540001170B5160004AA1488D2
:1040D00005AA15784A685078117800022A4A0843E0
:1040E000801805284BD807F02FFE03131E29343FF4
:1040F0000720032C0BD80422121BAA4200D92A0045
:1041000022491A803000091907F0A6FD002070BD71
:104110000720112CFBD81222121BAA4200D92A0018
:104120001B491A80EEE707200E2CF0D80F22121B35
:10413000AA4200D92A0017491A80E3E70720032C76
:10414000E5D80422121BAA4200D92A0012491A807B
:10415000D8E70720032CDAD80422121BAA4200D980
:104160002A000E491A80CDE70720032CCFD804225D
:10417000121BAA4200D92A0009491A80C2E700226C
:104180000A201A80C3E7C046DCD5FFFF83BE0011BA
:10419000EC61FF1F73BE00116EBE001169BE0011FD
:1041A00064BE001110B50D21024A034806F050FD0F
:1041B00010BDC04658BE00115C41FF1F13B5104C26
:1041C0000423217C01AA00F0ADF9002815D16B462B
:1041D0009A88236852BA92B25343228909491B0C28
:1041E0009B184B806B46DA88636852BA92B253438D
:1041F00062891B0C9B188B8016BD0120FCE7C04612
:104200000062FF1F1862FF1F13B5124C06236A4697
:10421000217C00F087F9002819D16B4619882368A2
:1042200049BA89B24B4321890B4A1B0C5B18538056
:104230006B46D97803335B781B020B435BBA61682A
:104240009BB24B4361891B0C5B18938016BD012008
:10425000FCE7C0460062FF1F1862FF1F37B5174C0E
:1042600007236A46217C00F05DF9002824D16B46C3
:104270001B787F2B20D86B46DD78F0232A041B03A4
:104280001A406B469B880E495BBA9BB21A4323685F
:104290002D09534322891B0C9B184B806B465A787F
:1042A0009B7812031B011A4363682A4353436289B4
:1042B0001B0C9B188B803EBD0120FCE70062FF1F9A
:1042C0001862FF1F7FB50226154C0022217C03AB2C
:1042D0000096050000F0F8F8002802D0012004B094
:1042E00070BD0E23217C0122280000966B4400F053
:1042F000EBF80028F2D16B469A892368D2BA53436F
:10430000228908491B149B184B806B46DA89636825
:1043100052BA92B2534362891B0C9B188B80DEE722
:104320000062FF1F1862FF1F70B5184C237C002B22
:104330000FD0382B0ED1164D280000F073F8CC2387
:10434000AC222800217C9B0100F027F9280000F016
:10435000A7F870BDE3890F4A934209D10C4D28009C
:1043600000F060F800222800217C00F005F9EDE75C
:10437000094A9342EDD1064D280000F053F89022EF
:104380002800217C920100F026F9DFE70062FF1F80
:104390003442FF1F830500008320000070B5144CD9
:1043A000237C002B1FD06369002B1CD0114D2800EB
:1043B00000F038F86369280098470400280000F0EE
:1043C0006FF8002C10D10C4B0422995E002905DAFD
:1043D0009C801A8801321A80200070BD074A9142E1
:1043E000F7DD9A80F5E70124FEF782FEF4E7C04688
:1043F0000062FF1F3442FF1F1862FF1F0F270000DB
:1044000010B58024064AA4001168436B234205D1ED
:1044100013685B1A032BF8D9012010BD0020FCE7BC
:104420006008FF1F70B5C17905000C00631E9C4138
:104430001A4BE402E41849000460C9B2007906F09E
:10444000F1F8E979687949000131C9B206F0EAF872
:10445000E8790930C0B207F04FFB0023E36661330F
:104460002360AA795B3B002A0ED022689A43023B64
:10447000134323600A23E36107332362002323638A
:10448000A3630133E36370BD22689A43022313439D
:104490002360462363610633A361EFE700500040C9
:1044A00070B5002504000368DD66C0790930C0B22C
:1044B00007F05AFC2900207906F050F829006079AD
:1044C00006F04CF870BD0000F8B51E0006AB1D7874
:1044D000002304681700E366616007F0F5FB012321
:1044E0008022E3662B0027615200013B08D207F0CF
:1044F000D3F908200A4A1168002D03D12800F8BD1D
:104500002261F2E7236F034203D02369013D337038
:10451000013613685B1A032BEED90125EEE7C0467E
:104520006008FF1F70B51C00002305681600EB66CD
:10453000696007F0C9FB01238022EB66230052006B
:10454000013B08D207F0A8F908200A4A1168002C9C
:1045500003D1200070BD2A61F2E72B6F034203D024
:104560002B69013C3370013613685B1A032BEED9BB
:104570000124EEE76008FF1F002370B504681500F2
:10458000E366616007F0A0FB0123E366256107F0A5
:1045900083F92000FFF734FF70BD70B51D000023C4
:1045A00004681600E366616007F08EFB0123E36692
:1045B00026610F33626B1A42FCD02B0A2361102351
:1045C000626B1A42FCD0EDB2256107F065F920005C
:1045D000FFF716FF70BD002370B504681500E36691
:1045E000616007F071FB0123E3662B0A236110234E
:1045F000626B1A42FCD0EDB2256107F04DF9200044
:10460000FFF7FEFE70BD70B51E00002305681400A4
:10461000EB66696007F058FB0123A619EB660F33C0
:10462000B44205D107F038F92800FFF7E9FE70BD64
:1046300021782961696B1942FCD00134F0E7000050
:1046400010B5084CE368002B08D18022064B5202BB
:104650001B689B186360054B1B68236007F0F4FA26
:10466000A06010BD4062FF1FC8F00040CCF00040C9
:1046700070B5184A936A916A9942FBD116498A68C3
:104680009A421FD39A1A8B60144B0126186893B272
:10469000D202D20E4343424300204C681B0A1B192E
:1046A00012029B180E4C0A684B60551CA3420CD892
:1046B000002801D04B600A600A4A136008680A4B60
:1046C000186070BD581E821ADDE7084A30009B183A
:1046D0002A00EAE700F000404062FF1F140AFF1FB3
:1046E00040420F00C8F00040CCF00040C0BDF0FFD9
:1046F00070B51F4C23793F2B01D93F2323711D4BEC
:1047000022791A701878C0B207F0F6F818231A49FF
:104710001A4A0B801A4913800B805380A3791949D8
:1047200080200B800C21938001334B43164D191CC4
:104730000001834200D9011C2980D1806379002BBC
:1047400001D101336371237A012B01D80223237233
:104750006279237A0D4853430A21584307F064F8DD
:104760000B4D2860E379052B01D81023E37170BD50
:104770003462FF1F480AFF1F4E42FF1F1C44FF1FE9
:104780004C42FF1F4A42FF1F4842FF1F71020000B8
:104790002462FF1FF8B520210020FEF761FE114CB6
:1047A000011E114D09D10C22104BC1CBC1C42800F0
:1047B00007F0B2FAFFF79CFFF8BD0C2220000C496D
:1047C000FEF722FE0C2802D0084B43CB43C40C2238
:1047D00028000849FEF718FE0C28EBD00C22002117
:1047E000E5E7C0463462FF1F0062FF1FE0BE001114
:1047F000FC0C0000F50C0000F0B51D4C8022A54417
:104800000400882069465201400507F015F89022FF
:1048100012016A441300200032C832C316C816C3FE
:104820008023144C144FA6689B033343A3603B6062
:1048300007F092FA8823A0685B05C01807F06CF8AF
:104840000025882329008022A0685B05C018401934
:104850006944520007F068FA80230135FF355B0197
:104860009D42EED1A6603E60044B9D44F0BDC04623
:10487000FCEFFFFF8C43FF1F9808FF1F0410000090
:10488000F0B5040087B0002825D0684607F09CF9F1
:104890001B4C022806D106226946200007F0B4F915
:1048A000002816D06946002301250F262F00E25C60
:1048B000013310091030874038002F0032409740F4
:1048C0003A0002434A610439062BEFD16846FFF7EC
:1048D00093FF07B0F0BD182269460A4806F0ACFF06
:1048E0006A46A300D358013305D01822FF21684639
:1048F00007F012FAEAE70134062CF1D1E9E7C046E5
:104900006509FF1F00090011F0B5002504000E0025
:1049100085B0AA4200D186E04B1C087801934B7801
:104920008978377909021943F3783F061B040B4352
:104930001F43039720706570252800D196E033D877
:10494000112813D807F050F969002F012F012F010A
:104950002F01AA00B800B1002F012F012F012F0154
:104960002F012F012F012F010F012901232800D131
:10497000E8E0DB2800D038E1042A00D8B1E01025B7
:10498000052A05D0551F2A003800711D07F064F96B
:1049900005223100200007F05FF92A003900601D70
:1049A00007F05AF905353EE0562859D010D833287B
:1049B00000D1A7E0552839D02628DAD1A14B29000B
:1049C000132218001D0007F0A7F9FEF791FB5CE029
:1049D000712800D177E0722800D189E0602800D1E9
:1049E00095E0DC28C5D1022A00D87AE07378BFB2FE
:1049F0006370B378A370032A05D0033A390092B2EA
:104A0000F01CFEF73BFC10223900E01CFEF7FCFC1A
:104A1000C51C002807DA607070E00C2220008A496B
:104A200007F01AF90C25280005B0F0BD013A874DB2
:104A30000C2A13D8002A0AD02800019907F00CF993
:104A4000FFF756FE0C2228008149FEF717FC2900CB
:104A50000C22601C07F000F90D25E4E70C22EBE7BF
:104A60007A4D7C4B2A0043CB43C2E9E7013A754DAE
:104A70000C2A11D8002A08D00199280007F0ECF878
:104A80000C2228007449FEF7F9FB29001322601C50
:104A900007F0E2F81425C6E70C22EDE706226F497D
:104AA000601C07F0D9F80625BDE712226C49601C8E
:104AB00007F0D2F81325B6E708226A49601C07F010
:104AC000CBF80925AFE7012A0ED07178F02908D874
:104AD000654D288801F0C6FD644B2A885200D35AE0
:104AE00000E0FF23637009E05F4A604B1288F5E73E
:104AF0005F4B012A04D072789A706270022592E7A7
:104B00009B78EFE72000FFF79DFA05008BE7013A5D
:104B1000574B584D062A10D8002A10D001212800E2
:104B20005970019907F098F801F058F82900062209
:104B3000601C07F091F8072575E70622EEE70022D2
:104B40005A70F3E7042A04D94B4D2F6007F07CF824
:104B5000A860FFF78DFD0422039003A9601C07F0F5
:104B60007BF805255FE7454D062ADFD90622280098
:104B7000019907F049F80028D8D0062201992800A9
:104B800007F06AF806223E492800FEF777FB01236A
:104B9000374A91780B439370C8E7012AA1D0707807
:104BA000FFF76EFEAAE7012800D0E2E6931E354F1C
:104BB000132B06D87378002B0BD100F017F900F0F7
:104BC0004DF9314B39001D78601C6A1E07F044F81E
:104BD00029E7551E2A000199380007F03DF83800F2
:104BE0002A49AAB2FEF74AFBE9E7DA281DD1042ACE
:104BF00000D876E7082A15D9B37972791B021343D6
:104C0000F27912041A43337A1B0613433B603B6864
:104C1000052231002000039307F01EF80422601DD6
:104C200003A94CE7FE236370F1E7DE2800D058E7C4
:104C3000511E012A01D10025F5E6019800F0B4FFCC
:104C4000F9E7C0460062FF1FECBE00113462FF1F8F
:104C5000FC0C0000E0BE0011F50C00000C62FF1F10
:104C6000EC61FF1F9043FF1F5042FF1FA864FF1F0E
:104C70003062FF1FED42FF1F4062FF1F6509FF1FEB
:104C8000ADAC00003164FF1F2F64FF1FAEDE0000DB
:104C900070477047020010B5094B0A32094C92B2B6
:104CA000DA815A8298811882207802F041FB04222E
:104CB000054B012120781A7007F00EF810BDC04690
:104CC0001A43FF1F7A64FF1F7964FF1F013870B514
:104CD000042809D807F038F8030928081200234BE4
:104CE0000221187806F0F8FF70BD204B08211878D3
:104CF00006F0B2FD00221E4B1A72F5E78022002456
:104D00001B4B1A4D52001A8108211A682878DC7250
:104D100006F072FF2100287806F0FEFE012000F068
:104D20007BFE00F05BFFDFE7104B0821187806F0F0
:104D300093FD1048FFF724F80F4B104A9B79002091
:104D400093800F4A13808022094B5200D8721A8137
:104D500000F062FE00F042FF0A4B9B78002BC3D0AC
:104D6000094A136006F010FEBEE7C0465062FF1FFE
:104D70002462FF1F5942FF1F3462FF1F1C44FF1FA4
:104D80004A42FF1F3062FF1F34F0004010B5002977
:104D90000BD1082809D1054B1B78002B05D0262202
:104DA000034B04485A72FFF775FF10BD5264FF1F92
:104DB0002462FF1FC40900000300F0B50A4D8E18DD
:104DC000B14202D152008018F0BD0C782F6824093E
:104DD0003C5D0F271C700C7801313C402F683C5D16
:104DE0005C700233ECE7C0464442FF1F0D22124BB9
:104DF00010B51A700C23114C11492370093A033B6A
:104E00001048637006F028FF2D2301220E490F4839
:104E1000A371FFF7D1FF01220D49FFF7CDFF01225A
:104E20000C49FFF7C9FF030000200B49020018706E
:104E3000FEF724FA10BDC0464E64FF1F2F64FF1F0B
:104E400083BE00113164FF1F6709FF1F3664FF1F17
:104E50006609FF1F6509FF1FAEDE000070B5134C29
:104E6000142220001249FEF7CFFA431E114D132BD6
:104E700019D8AB78002B16D0431C2B7009236B700C
:104E800000230019037028780B4B01302900C0B2B1
:104E9000187006F069FC297822000139C9B2002097
:104EA00005F0F4FD70BDFFF7A1FFECE73164FF1FD3
:104EB000AEDE00002F64FF1F4E64FF1F10B5114BC4
:104EC0001A781870002A0ED000280BD10E4B1A78D1
:104ED000062A07D85423D340DB0703D50B4B187899
:104EE00002F026FA10BD0028FCD0074B1B78012BDE
:104EF00002D0033B022BF5D8044B0121187806F0B1
:104F0000EBFEEFE75264FF1F7964FF1F7A64FF1F17
:104F100070B5514E514A52493070082005F042FC9C
:104F20000121022005F048FB022005F029FC0121A7
:104F3000002005F041FB002005F022FC00F0D2FE2D
:104F4000FEF7D6F806F028FF032246494648FFF749
:104F500033FF2D24030004221C7044490130FFF765
:104F60002BFF30230470424D424C437083702E3B24
:104F7000062220004049EB87FEF746FA062813D0A8
:104F8000200006F021FE022809D00321200006F0AF
:104F90007BFD8D23E3706E3B237119336371062211
:104FA00020003549FEF76AF9344B1B68FC335C641A
:104FB000FFF754FF0020FFF781FF314C314A0121F8
:104FC000314B1278207802F075F9304A304B127864
:104FD0000021207802F06EF901222E4B1A702E4B20
:104FE000DB78552B31D12D4B3B325A722C4B2D4A4D
:104FF000AB81EA812B826A822021307806F00CFC9A
:105000000120404205F08EFD0120404205F02AFEBD
:10501000FFF7C8F8FEF77CFE00F0B2FC012040422A
:10502000FEF752FF012006F0D7FBF02001F0FEFA58
:105030000121307806F050FE307802F0D5FA1A4897
:1050400006F022FEFEF712FD70BD6422174B5B795D
:1050500053431A000A32CBE75062FF1F8D4D0011F7
:10506000914C00119043FF1FEC61FF1F0C62FF1F6A
:105070001A43FF1F6509FF1FADAC0000A464FF1FAA
:105080007A64FF1F7842FF1F5942FF1F4E64FF1FC3
:105090002F64FF1F2064FF1F3062FF1F2462FF1F69
:1050A000C4090000CE0900005262FF1F3462FF1FD6
:1050B000F8B50A0020230D001A40194263D05E4B58
:1050C0001B78002B5CD0FFF7D3FA5C4B5C4C5D4E39
:1050D00099686268737A8A1ADB039A4202D3616024
:1050E000FEF7C4FC327A217A531EDBB2994205D115
:1050F000FFF71AF9002000F0A7FD15E09142F9D35F
:1051000000272772FFF74AF9A37ABB4202D0A772A1
:10511000FEF73AFD012000F097FD4B4F3800FEF7F7
:105120002FFE390006F008FC637A002B25D0013BE6
:10513000DBB26372002B20D1444BDB78552B01D1BD
:1051400006F022FCE37A002B12D00023A27AE3724D
:105150009A4202D0A372FEF717FD3D4A3A4F1388D8
:10516000380001331380FEF70BFE390006F0E4FB34
:10517000642370795843FFF78DFD237A013323723E
:1051800020206840F8BD0BB2002B0ADA314B1878AA
:1051900006F0F2FD002801D006F0B6FD80200002E6
:1051A000EFE70224214206D0254B01201A72FFF7B7
:1051B00085FE2000E5E70B071ED5FFF759FA1F4BC8
:1051C0001F49204C98684A68637A821ADB039A4226
:1051D00002D34860FEF74AFCFFF7E0F8FFF7A4F8B7
:1051E000012000F031FD00F0E5FB2368DB0701D56D
:1051F000FEF762FF0820C4E7CB0609D5FEF7C4FC22
:105200000D4B1B78002B01D1FEF796FD1020B8E75F
:105210000124214207D0104800F06CF806F024FC6D
:1052200000F0F8FCC5E70424080020402142A9D082
:10523000FEF766FEBDE7C0465264FF1F4062FF1FD7
:105240002462FF1F3462FF1F5942FF1F3062FF1F9D
:105250001862FF1F5062FF1F3C42FF1FF0B51B4B3F
:105260001B4F1B883A8804001A4E1B4D85B09A428A
:105270000DD832889A420AD3184B1A882B889A4242
:1052800005D1174A174B12881B889A421BD005205C
:1052900001F022FA3B8802AA1380338801905380E0
:1052A0002B88114D93800F4B02A91B88D3800F4B85
:1052B0002A78188802F03EFF0D4B08212878019AC1
:1052C0001C7006F079FD05B0F0BDC0461E64FF1FDE
:1052D0004E42FF1F4C42FF1F4A42FF1F1C64FF1F2C
:1052E0001A64FF1F4842FF1F7A64FF1F5042FF1FCE
:1052F0001864FF1F13B50C4B1C78002C11D100282B
:1053000001D00A4B18600A4A0A4B11780A4A1078F1
:105310000A4A01920A4A0092002205F0AFFA2000E0
:1053200016BD1124FBE7C0467964FF1F1464FF1FFC
:105330007864FF1F6864FF1F7A64FF1F5464FF1FB7
:105340005864FF1F10B5064B12201B78052B06D1A1
:10535000044B13221988044B187801F099FB10BDF7
:105360007964FF1F5042FF1F7A64FF1F10B50024AD
:105370000122114B52421870104B1C70104B1A80B6
:1053800002F032F904220F4B21001A700E480C3241
:1053900006F02AFA102221000C4806F025FA07220E
:1053A0000B4B1C600B4B1C700B4B1C700B4B1A7087
:1053B0000B4B1C7010BDC0467A64FF1F7964FF1F41
:1053C0005042FF1F7864FF1F6864FF1F5864FF1F6F
:1053D0005464FF1F2E64FF1F2D64FF1F5242FF1FE6
:1053E0002C64FF1FF8B5174C0600257806A8142476
:1053F0000078052D23D1B41F134FA5B21824BD4248
:105400001DD88D1FADB2BD4219D8FA256D00AA4234
:1054100015D21D000D4F0A3DADB2BD420FD80C4C48
:1054200026800C4C21800C4900240A800B4A1380F2
:10543000FFF714FF0A4B0421187806F00DFA20003C
:10544000F8BDC0467964FF1F790C0000750C0000A0
:105450004E42FF1F4C42FF1F4A42FF1F4842FF1FA0
:105460007A64FF1FF0B50BB20D0089B0002B00DB92
:1054700070E1A44E307806F07FFC041E50D0037813
:10548000A22B00D122E1D02B1AD0912B45D1437809
:105490000E2B42D19C4B82889A423ED19B4A836814
:1054A0001278052A39D1032018567F2835D0984B19
:1054B0001B68002B31D05B68002B2ED098472CE066
:1054C0008078072829D806F03FFC0428183F3F744D
:1054D000A8D86378002B0CD101218C4B19708D4B0F
:1054E0001A78002A5BD08C4B307801F0E3FE00285C
:1054F00055D00722854B1A7051E061780029F8D108
:10550000E378002B11D0854A854B1278307801F072
:10551000D1FE60706378002BEBD1200006F0F4FB25
:1055200080200002684009B0F0BD784B1B78022B48
:10553000F3D00121307806F03FF90028EAD10121AB
:10554000307806F0C9FBE5E76378002BD1D16F4FC7
:10555000032807D13B78052B02D101333B701EE0B5
:105560000223FBE76F4B1A886F4B0293002A0BD084
:105570001B78002B03D00121307806F01DFC3B780E
:10558000062B04D1013BE9E7029B1A70F7E7042BD5
:1055900041D10121029B3078197006F09DFB5C4BD4
:1055A0001B68002BB9D01B68002BB6D0574A107867
:1055B00084E76378554F002B27D10622211D5B48D5
:1055C00006F04AFB62895A4B5A491A80A2895A4B03
:1055D0001A80E3890B800521397058490A80584A9E
:1055E0001380228A574B1A80574B1B78012B09D105
:1055F0001F2001F071F8FA22920042430421307812
:1056000006F0DAFB0022484B75E7312B00D070E73B
:105610000022454B1A700323A0E7062200214348CD
:1056200006F0E2F80023454A04211380444A30780A
:105630001380444A138006F00FF90821307806F0F1
:105640000BF9A379083B5A425341304A0333137094
:10565000304B1B78002B06D0334B30781A78002A59
:1056600006D001F065FE0122314B52421A8096E7C6
:105670000121197006F030FBF5E70821307806F0BB
:10568000EBF86378002B00D047E72C4B2D4F0293AB
:10569000E388029A04211380294B307803932389ED
:1056A000039A138063893B8006F086F8002800D0B7
:1056B00033E7264B1B68002B00D12EE70399029895
:1056C0003A88098800881B68984726E74379132B96
:1056D00000D022E70389012B0AD11D4B1B78022B36
:1056E00006D10821307806F0B7F8FFF72BFE14E753
:1056F000052000F0F1FF08210200307806F05CFB85
:105700000BE7C0467A64FF1F051400007964FF1F91
:105710001464FF1F7842FF1F5942FF1F4E64FF1F92
:105720002F64FF1F5064FF1F5264FF1F2164FF1F7F
:105730005042FF1F2864FF1F2A64FF1F1E64FF1FC3
:105740001C64FF1F1A64FF1F2064FF1F1064FF1FEB
:105750001864FF1F8020C001014200D0E2E6CB07A1
:1057600031D5324B1B78002B1DD0314E05AC337830
:10577000052B1AD1023B23702E4B21001B7823727C
:105780002D4B1B7863722D4B187801F037FD0028E4
:1057900009D007202A4B30701B68002B03D01B68F0
:1057A000002B00D098470120BCE60E20254B062296
:1057B0001B7825492370254B1B78637002ABC018FA
:1057C00006F04AFAD8E7022308001840194209D027
:1057D000174B1B78052B03D11D4B188806F094F945
:1057E00002209FE60424214203D0FFF737FD20006A
:1057F00098E6082308001840194200D193E6154B9B
:105800001C78012C03D0022C0DD008208AE6124B04
:10581000124A134913481B8812880988008800948B
:10582000FFF7E0FDF1E7FFF78DFDEEE75264FF1FA4
:105830007964FF1F5242FF1F2C64FF1F7A64FF1F11
:105840001464FF1F2E64FF1F5342FF1F2D64FF1FB0
:105850005042FF1F1864FF1F4842FF1F4A42FF1FAC
:105860004C42FF1F4E42FF1F10B502A804880B20B8
:10587000002C10D1496808784978090201430C4886
:10588000814209D1022119800A4B59881170DB78B5
:1058900000205BB2537010BD074C0A20A142FAD120
:1058A00002211980034B998811705B79F0E7C0469B
:1058B0006E2A00001862FF1F6F2A0000F7B515005E
:1058C00008AA16884A680F4F1478527812022243A9
:1058D0000A24BA4214D10122DBB2019200962A00B6
:1058E00005F0D2FE041E0BD1074B1B68002B07D01E
:1058F00068782A78000210434242504101309847AC
:105900002000FEBD022900008C64FF1F30B5012578
:1059100003790400BFB02B4225D01449408805F01C
:105920001FFA28420CD0124B01A95B8D00220B807C
:1059300002234B800F4B5B888B80608802F0F0FA6B
:105940000D49608805F00CFAC0070CD50B4B01A976
:105950001B8800220B8002234B80064B9B888B8088
:10596000608802F0DDFA3FB030BDC0468464FF1F9E
:105970007C42FF1F1862FF1F7C64FF1FD642FF1F7F
:1059800010B5074C0749200005F0A0F92000064992
:1059900005F09CF90721054A054805F059F910BDA5
:1059A000FFFF00008464FF1F7C64FF1F0CBF001119
:1059B0007C42FF1F10B5024803F034F910BDC04609
:1059C0000D59001170B55F25082607498400CA7873
:1059D0008B7840012A40B3433440A8432343024319
:1059E0008B70CA7070BDC046ED42FF1F010043B20C
:1059F00004205A0002409B000C3003401A43152338
:105A000010B5044CE0789843143B0B401843024314
:105A1000E27010BDED42FF1F10B5054B0824197947
:105A20000A00A243002801D022000A431A7110BDC7
:105A3000ED42FF1F10B5054B4024D9780A00A24360
:105A4000002801D022000A43DA7010BDED42FF1F8A
:105A50000821F8B5324D334BAE7804000E40AE70DD
:105A6000984204DD67232B70473B6B70F8BD2E4BCB
:105A7000984203DAE0232B703A3BF6E700232B70C1
:105A80006B7083B21A0029485F3292B2284F82426B
:105A90002CD9002C03DA5B421CB204232B70053492
:105AA00020B20A2105F0C0FE04B2FA239B009C42FA
:105AB00032DB08232A7813432B706421200005F081
:105AC000B3FE0A2100B205F047FE09B22A787B5CDA
:105AD00013432B700A21200005F0A6FE0A2100B214
:105AE00005F03AFE09B27B5C6A780AE06970002C26
:105AF000DBDA5B421CB204232B70F3226B78092C97
:105B0000E8DC13436B700A21200005F025FE09B282
:105B10007B5C1E43AE70A9E7632CCEDCEDE7C0468C
:105B2000ED42FF1F1B4E00001DFCFFFF2A08000076
:105B300036BF00110823F7B5194FCD003E79040098
:105B40001E403E71EDB2632806DD5F3333433B7187
:105B500020231D437D71F7BD0300093305DA20239F
:105B60005B4233433B71A623F3E70E4B01930028BE
:105B70000BDA0423444224B23B710A21200005F0D1
:105B8000EBFD019B09B25B5CE3E70928F5DD0A2127
:105B900005F04AFE019B00B21B5C1E433E71ECE720
:105BA000ED42FF1F36BF0011F8B50A4F05003B78E4
:105BB0000E00002B0CD0084C2000FEF733FC330005
:105BC0002A0020003978FEF71EFD2000FEF768FC51
:105BD000F8BDC0469764FF1FF442FF1F70B50A4E20
:105BE0000A4D06223100280006F00EF8002809D0E0
:105BF000074C31000622280006F02EF8072120006D
:105C0000FFF7D2FF70BDC046ED42FF1F9164FF1F3A
:105C10009064FF1FE622402110B50A4B1A70403AEB
:105C20005A703E329A70DA780A40DA70082219798E
:105C30001140533A0A431A71F3225A71FFF7CEFF0B
:105C400010BDC046ED42FF1F10B5002838D0214CD2
:105C50000223E05E204B1B685B0632D5092332210C
:105C6000584305F0E1FD4130FF3000B2FFF7F0FE90
:105C70000520FFF7A7FE0422A35E184A6320934283
:105C800005DC32331800642105F0CEFD00B201219D
:105C9000FFF750FF237A0024132220009A4260412C
:105CA000C0B2FFF7C7FE2000FFF7A0FE0C4B18782C
:105CB000053843425841C0B2FFF7AEFEFFF78EFFF2
:105CC00010BD0A21053005F0AFFD00B2FFF7C0FEA0
:105CD0000320CEE71862FF1F3462FF1FDD2600009D
:105CE0007964FF1F70B500250A4C2000A571FEF7EE
:105CF00099FB10233E212000074AFEF784FCA842AE
:105D000000D13E35054B20001D70FEF7C9FB012375
:105D1000A37170BDF442FF1F26BF00119764FF1FDF
:105D20000200F0B501270A480A4E51188B1A002BC1
:105D300000DCF0BD08241578430868403840400076
:105D4000805B013C58406D08002CF5D10132EDE735
:105D5000FFFF000046BF0011F0B500250F269D4251
:105D600000DBF0BD4C5D070944403440A400A0585E
:105D700001357840F3E70000F0B589B06A460D00C0
:105D80000B000F27110010351C7801332600240961
:105D90003E40167054700232AB42F5D12023024AC5
:105DA000FFF7DAFF09B0F0BD4CBF0011F0B54E7837
:105DB0000B7889B036020C00170001901E43012AAF
:105DC00061D9954B9E4200D877E001339E421CD1A9
:105DD000062A17D1CA788B7812021A430B791B0452
:105DE00013434A7912061A438C4B5A6100221A70E7
:105DF0005A808B4A5A608B4A9A608B4ADA6000203C
:105E000009B0F0BD88225205EEE7884B9E423CD196
:105E100082498B78002B00D0F6E00C2A31D10F227A
:105E2000A3789343E27812021343227912041343B6
:105E30006279120613434B60E279A07912020243A1
:105E4000207A00041043627A12060243CA60E27AA2
:105E5000A07A1202024376484A81834208D804237A
:105E60006E49142201980B7005F0F6FE1420C7E766
:105E70001201D21889235B059A42F0D801238B7056
:105E8000BDE7022AFAD00523EAE76A4A01239642CF
:105E9000E6D1FFF757FA052F0CD9E378A2781B0259
:105EA0001343227912041A4363791B061343624A8F
:105EB0000393136005F068FDA1E7584D2B78002B84
:105EC0009DD1AB78002B00D1A0E02B8901339BB290
:105ED0000093B34200D091E0132AD4D9CF7C8B7CBD
:105EE0003F02122120001F43FFF71AFF874200D014
:105EF0008EE0002E3DD1E378A2781B021343227975
:105F0000E96812041A4363791B06134303930A22B8
:105F10008B4212D1FF23A370E370237163716B89ED
:105F2000002B09D1E37B227C1B0212041343A27BCA
:105F300013431B0901336B8100226B89002B8ED028
:105F4000002A67D1686837013818000B6B690003B5
:105F50000390984205D9686105F0DEFCEB780133C7
:105F6000EB7068681022A11C381805F0DDFE2E8148
:105F700045E76F89009A7B1E9BB293423AD1E27843
:105F8000A37812021A43237905A81B0413436279EC
:105F90006C6812061A43EB6800920392211D0C22D2
:105FA000049305F059FE0120260004A94042103652
:105FB000FFF7E2FE013F012F17D1009A0B23286162
:105FC000824200D04CE704221C49200005F0ACFEC0
:105FD000042203A9686805F02FFCE968039AFF23EF
:105FE000914200D13CE7F73B3AE73100FFF7C4FEAE
:105FF0001036DFE70923B742A4D831E7009BB3424C
:1060000000D9FCE607232BE7022329E7032327E730
:10601000062325E70A2323E7FFFE0000FC42FF1FBB
:1060200000000111FFFF00005048593601FF000039
:10603000FFFF001102FF000034F000400843FF1F83
:1060400010B5034C0B000122210000F06BFA10BDCB
:10605000016200110B8870B506000D000224162B9A
:1060600011D92B000322094900F05CFA041E0AD161
:10607000074B2A881B88191C934200D9111C300039
:1060800089B200F0EFFA200070BDC0462D62001109
:10609000AA64FF1F10B54A780400013A0B000220E1
:1060A000012A07D80A78002A04D0052220000249D4
:1060B00000F038FA10BDC0465B6200110A7810B5D6
:1060C0000B0004000220002A04D00722200002490D
:1060D00000F028FA10BDC046076300110A7810B519
:1060E0000B0004000220002A04D0092220000249EB
:1060F00000F018FA10BDC0466D63001110B5034CD6
:106100000B000B22210000F00DFA10BD9D63001161
:1061100010B5034C0B000D22210000F003FA10BD56
:106120000F64001110B5034C0B000F22210000F08A
:10613000F9F910BD696400110A7810B50B0004006C
:106140000220002A04D011222000024900F0EAF9BE
:1061500010BDC04679640011002310B51322190048
:1061600000F0E0F910BD000010B5034C0B00172241
:10617000210000F0D7F910BDCB640011002310B549
:106180001922190000F0CEF910BD000010B5034C23
:106190000B001B22210000F0C5F910BD05650011A0
:1061A000F7B584890D0006000121002C22D00023C0
:1061B0008268D3561778002B1EDA0C2C1AD90C3CA7
:1061C000A4B2131940880093230002F086FE431EF8
:1061D000984101307B06DB0F6B703F23013C1F4071
:1061E000A4B22870AF70AC80002C07D0B368013324
:1061F000AB6000210800FEBD0020EBE7AC60F8E7D3
:106200000B7803704B8843704B881B0A83700B79A3
:10621000C370042070470420022B06D1002053785D
:1062200011781B02009A0B43138070470B88037090
:106230000B881B0A43700220704704200099834298
:106240000AD1537810781B0203430B80D3789078DF
:106250001B02034300204B807047F8B50D004B78BC
:1062600001240021461C03702B788B4201D82000AA
:10627000F8BD6B78B01C4F1C012B10D18900691838
:106280004B88022233704B88B9001B0A737069185F
:1062900005F0EAFA04360434A4B2F9B2E4E71223B2
:1062A00059436B185A88043132705B8810221B0ADC
:1062B0007370691805F0D8FA12361234ECE770B52D
:1062C000049D14001E00052B01D8042070BD6378C6
:1062D00012781B0213432B80E378A2781B0213432E
:1062E00002226B802A71211D681D063E05F0BCFA52
:1062F000B2B22A81E92AE8D82800A11D0A3005F0A7
:10630000B3FA0020E2E7002310B50A789A4201D8D8
:10631000900010BD9A008A18548801330470548884
:10632000DBB2240A4470948884709288120AC27086
:106330000430EAE710B51100029C062B04D00420BB
:106340001022142B01D010BD022222714B78087844
:106350001B0203432380CB7888781B0203436380AE
:106360000431601D05F080FA0020ECE710B50C78D0
:106370008B7804315C43E4B203702200013005F0F5
:1063800073FA601C10BD0420022B06D10020537844
:1063900011781B02009A0B431380704710B50C0054
:1063A0000A88023105F060FA208810BD70B504003B
:1063B0000D0004981100012B01D8042070BD16783F
:1063C00052781202324302800200F132557014708A
:1063D000E125002C00D10C35023B9AB24280AA4242
:1063E000EBD80231043005F03FFA0020E6E7042044
:1063F000009983420AD1537810781B0203430B8023
:10640000D37890781B02034300204B80704710B56F
:106410000C000A88023105F027FA208810BD000020
:1064200070B501211E000420049C0E400B4218D1BF
:10643000CB40DDB28D4214D90A49DBB209889942BA
:106440000FD32300EE331D70330058001118497824
:10645000165C0902314301332152D9B28D42F4D87E
:10646000002070BD1443FF1F10B50C000A880231D4
:1064700005F0FAF9208810BD10B50C788B7804313E
:106480005C43E4B203702200013005F0EDF9601CBA
:1064900010BD10B511000298032B01D8042010BDC7
:1064A00014785278043B120222430280CA788C7816
:1064B0001202224342809AB28280EB2AEED8043143
:1064C000063005F0D1F90020E9E710B50C000B8883
:1064D00003700B881B0A43704B8883704B881B0A20
:1064E000C3708A880430063105F0BEF9A0880430F4
:1064F00080B210BD0420012B03D100201378009A34
:106500001370704710B50C000B8803700B881B0AC2
:1065100043704A880230043105F0A6F960880230E1
:1065200080B210BDF0B589B003931E4B02924200B9
:106530000700D05A019102F020F81325061E2DD035
:10654000029B01240370019B002B04D000190399C6
:106550009847001984B26B461B7A5BB2002B0FDAA6
:106560001021380002F01CFB1925002813D130003F
:106570003219E1B202F066FC051E0CD10C34A4B253
:10658000042304AA380005A993800696948101F09B
:10659000AFFD051E02D0300005F06EFB280009B0EB
:1065A000F0BDC046A864FF1F70B505000C000028B0
:1065B0000CD00020814209D010222000044905F0AF
:1065C00053F901202B7823736B78637370BDC04639
:1065D0008CBF0011F0B506000D0017001C0085B03F
:1065E00002291BD00020102907D1022B07D0102B25
:1065F00003D115E00020102C08D005B0F0BD69468D
:106600003800FFF7D1FF2A0069460BE069463000E9
:10661000FFF7CAFF22006946380004E0022BE9D1E7
:106620002A003900300005F057FAE6E7031CF0288D
:1066300000D9F023032008499AB2013A0B80D317FE
:10664000034006499B189B100B80D30F04499B18ED
:106650005B100B807047C0461843FF1F1643FF1F97
:106660001443FF1F034B1B888B4202D3024B400095
:10667000C15270471843FF1FA864FF1F014B400021
:10668000185A7047A864FF1F1722014B1A807047E1
:10669000A864FF1F70B505000E2005F045F9041E23
:1066A00013D0D0230370002306228370074945705E
:1066B000033005F0D9F8064B2100DA8A62811B7E8F
:1066C0002373044B187805F03FFA70BDC464FF1FB4
:1066D000B464FF1F6843FF1F262803D8024B400005
:1066E000C05A70470148FCE71A43FF1FFFFF000034
:1066F00070B506000C00094D1C220021280005F091
:1067000073F8074B1E70074B1C7005F045F9012309
:10671000002801D0002312202B7070BDB464FF1F2D
:106720006843FF1FD564FF1F70B505000D4C0800BE
:10673000E260A16010220021656005F0BDF901282A
:1067400003D11021A06802F058FD1022002128007A
:1067500005F0B2F9012803D11021606802F04DFD67
:1067600070BDC046B464FF1F70B5041E05D100297A
:1067700003D006220D4805F077F80D4B1D78012D4A
:1067800011D1002C05D102221A7005F045F928001C
:1067900070BD00221A70074B1B78FF2BF7D020002A
:1067A000FFF778FFF3E70025F1E7C046C464FF1F59
:1067B000B464FF1F6843FF1F030010B5002801D118
:1067C000002010BD00780B4A002803D15988D182DF
:1067D0001B7913761378022BF2D10023984200D153
:1067E00003331370044B1B78FF2B01D0FFF752FFCC
:1067F0000120E6E7B464FF1F6843FF1F002911D0A2
:1068000000280CD04B79012803D140225242134377
:1068100003E03F221340032802D001204B71704750
:106820004022F4E70800FAE770B5094D0100287826
:1068300000280BD0074C0622200005F015F8210097
:106840002878FFF7DBFF200004F0A6FF70BDC046EC
:10685000D464FF1FAE64FF1F00290AD0012808D1AD
:106860003F224B799343C02B03D0403B5A425341C4
:10687000981C704770B5174D06002B78FF2B15D06C
:106880000A2005F051F8041E10D0D0230370C83B35
:106890008370114B11491B784670C3700622043077
:1068A00004F0E2FF2100287805F04EF90C4B1B782C
:1068B000012B0DD10B4B1B68002B03D09B68002BC9
:1068C00000D09847084B04211878084A05F094F93D
:1068D00070BDC0466843FF1FD464FF1FAE64FF1F36
:1068E000D064FF1FFC64FF1F0065FF1F60EA00000B
:1068F000014B98687047C046B464FF1F014BDB68CA
:1069000018687047B464FF1F074B10B5DA68136846
:1069100001331360054B1878FF2803D08021C9018B
:1069200005F0DAF910BDC046B464FF1F6843FF1FCD
:10693000F7B50E0002F0C8F8051E1CD00E4B06621B
:106940001F78002F00D10778AB791020019304F055
:10695000EBFF041E0FD0D0230380C73B8370019B45
:10696000E91DC3700622043004F07EFF21003800C8
:10697000E66005F0E9F8F7BD6643FF1F014B1878A4
:106980007047C046D464FF1F054B002805D1054B56
:106990001A78054B002A00D1014B18007047C046F9
:1069A000C464FF1FD464FF1FAE64FF1F014B58680F
:1069B0007047C046B464FF1F024B1868431E9841DD
:1069C000C0B27047D864FF1F421E03000120152A81
:1069D00003D9FF3B5A425341D8B27047F0B51C006F
:1069E00000230E0085B0039002920B70029A93422E
:1069F00001D3002019E0E55C5A1CD2B2002DF8D07A
:106A0000029851198142F4DC0233DFB2A35C180012
:106A10000193FFF7D9FF002807D0013D019A0399A0
:106A2000EBB233708A4202D1E01905B0F0BDDB1938
:106A3000DBB2DBE710B50C0002F09EF80300122079
:106A4000002B03D02100588804F096FE10BD0000F2
:106A500070B50E4D84006359002B15D0186A0028BC
:106A600001D005F021F82B59586A002801D005F013
:106A70001BF82B59986A002801D005F015F8285901
:106A800005F012F800232B5170BDC046E464FF1FCF
:106A90001C4B70B504000E00150099420AD11A4B28
:106AA0001B68002B01D1122070BD1B68002BFAD08F
:106AB0009847F9E7154B994215D1134B1B68002BEA
:106AC0000AD01B68002B07D09847002804D1104B30
:106AD0001C70104B1D70E7E729002000FFF7AAFF8C
:106AE0000028E1D1F3E7080001F0EEFF0028DAD03A
:106AF00003780320A342D7D12900300004F03CFEE4
:106B0000D2E7C046FEFF0000E064FF1FFFFF000069
:106B1000DD64FF1FDC64FF1FF7B50400808801F00F
:106B2000D3FF0025A84203D00578A08802F008F81A
:106B30001C4E3378002B1FD0AB421DD11A4B2800BE
:106B40001978FFF777FF002818D000233370A37956
:106B50000820A778A688019304F0E6FE011E0DD058
:106B6000D0230370CA3B8370019B4770868083717A
:106B7000280004F0E9FF01E0002DE8D1A0880B4BCC
:106B80008200D358002B01D0FFF762FF1721A088A5
:106B9000FFF768FDA08801F027FDA08801F0FEFD49
:106BA000F7BDC046DD64FF1FDC64FF1FE464FF1F08
:106BB000F0B587B01D000CAB1B88070001930DAB2F
:106BC0001B88142002930EAB1B88160003930FAB97
:106BD0001B880091049310AB1B88059304F0A4FE5E
:106BE000041E1AD0D0230370CB3B47708370C6704D
:106BF000062229000430002D11D004F035FE019B3F
:106C000021006381029B0098A381039BE381049B85
:106C10002382059BA37404F097FF07B0F0BD04F036
:106C2000E3FDECE7F7B5009308AB1B8807000C20E9
:106C30000D001600019304F077FE041E13D0280007
:106C400001F042FF00280FD00078D0232370C93B09
:106C5000A370009B21002381019B6770A580E680C3
:106C6000638104F071FFF7BD014B1878EDE7C04672
:106C70006843FF1F13B5040064890389C2888188B3
:106C8000C0780094FFF7CEFF13BD000010B5044C90
:106C90002068002803D004F007FF0023236010BD04
:106CA000E864FF1FA122F0B5818892004A43384B67
:106CB000384F1B6804009B189D2292009B18827914
:106CC00089B01A603B68002B5FD01D78324B1B687F
:106CD000002B04D05B68002B01D0002098472600D1
:106CE00008363100E079FFF7B7FD237DE07102003F
:106CF000E0780493638A29000393238A0293E3894B
:106D00000193A38800933300FFF752FFE378002B31
:106D10000BD1E289A379A18802920196E279280039
:106D20000092012201F0DAFEE0703B68002B20D0D7
:106D3000FFF7ACFF194D287800281AD0184B1978A6
:106D4000FFF778FE002814D02B78E6780820079308
:106D5000A78804F0E9FD011E09D0D0230370CA3BC7
:106D60004670837087808671079804F0EDFE0023DB
:106D70002B701721A088FFF775FCA08801F034FC68
:106D8000A08801F00BFD09B0F0BD064B9DE7C046A1
:106D90003409FF1FE864FF1FFC64FF1FDD64FF1F51
:106DA000DC64FF1F6843FF1FF8B5070008000E00F2
:106DB00001F08AFE041E18D02620FFF78DFC051E68
:106DC00000D12578062004F0AFFD041E0DD000216F
:106DD000062204F009FDD0232370C23B2100677016
:106DE000A370A680E8B204F0AFFEF8BDF0B585B0A0
:106DF00001930AAB1B78070002930BAB1B780800CA
:106E00000D000092039301F05FFE061E22D01020B9
:106E100004F08AFD041E1DD01022002104F0E4FCC1
:106E20002620FFF759FC002800D13078D0232370AA
:106E3000C13BA370009B21002372019B67706372AA
:106E4000029BA580A372039BC0B2E3720C9BE3601C
:106E500004F07AFE05B0F0BDF7B50D00019001F029
:106E600033FE071E20D00E2004F05EFD041E1BD052
:106E70002620FFF731FC061E00D13E78D023238068
:106E8000C53B0622A370F91DE01C04F0EDFC019B3C
:106E90002A0063810123DD401A401D402100227336
:106EA0006573F0B204F050FEF7BD0000F0B585B098
:106EB000029010000D0017000A9E039301F004FEDB
:106EC000041E31D0029B002B2ED1039B02795B075D
:106ED00024D5122313430422002E08D10B99002934
:106EE00005D10C99002902D10D9900291AD01A4315
:106EF0000D9B2271002B00D0C9E0002E00D1CFE005
:106F0000002D00D0CCE0606A002801D004F0CCFD58
:106F10001C21300004F078FD606205E002239A43F2
:106F20000E33D7E793432371654BBA00D458002C36
:106F300000D1AAE0002E10D0236A002B03D11C2020
:106F400004F0D2FE20625E4BBA00D358186A0028C3
:106F500003D01C22310004F087FC0C9B002B12D0C4
:106F6000574CBB001D596B6A002B03D1162004F04F
:106F7000BBFE6862BB00E358586A002803D01622A3
:106F80000C9904F071FC0D9B002B11D04C4DBC00F2
:106F90006659B36A002B03D1142004F0A5FEB06239
:106FA0002B59986A002803D014220D9904F05CFC38
:106FB000380001F089FD051E67D0414BBA00D35857
:106FC000002B62D01A6A3420002A00D11C389A6A39
:106FD000002A01D0143080B20B9A002A01D01C3054
:106FE00080B25B6A002B01D0163080B204F09CFCAA
:106FF000041E4AD01822002104F0F6FB2620FFF7D9
:107000006BFB0190002801D12B780193D0232370D2
:10701000029B200063700A23294EA370039BBD00CE
:10702000A371AB59A780196A1830002905D01C221A
:10703000A06004F019FC200034307359996A0029CB
:1070400007D0030014221433E060029304F00CFC18
:1070500002980B9B002B08D003001C221C330B99B9
:107060002061029304F000FC02987359596A0029C8
:1070700003D01622606104F0F7FB6B4621001879FB
:1070800004F062FD3800FFF7E3FC05B0F0BD10220C
:107090000D9B0D991B69A018236204F0E5FB2CE7FA
:1070A0000B9B002B00D13FE7012D00D03CE7606A2D
:1070B000002801D004F0F8FC1C210B982AE7C046F8
:1070C000E464FF1F10B5044C2068002803D004F0CE
:1070D000EBFC0023236010BDD864FF1F0B4B07B5EA
:1070E0001A68002A01D100200EBD6946531C0120F8
:1070F00012780731FFF772FC0028F4D002780123E0
:10710000100018401A42EED0EEE7C046F464FF1FAC
:10711000F0B51F4F01203B6887B0002B25D09B782E
:10712000059300F0B3FB002821D00A20FFF7D4FA22
:1071300004000B20FFF7D0FA164B05001E78731ED3
:107140009E413B68F6B2191DD878FFF757FB3B68A4
:107150002900DA7A043303929A790193029200901B
:1071600033002000059A04F007FC07B0F0BDFFF7DC
:10717000B5FF002805D00620FFF7AEFA040007206F
:10718000D8E70820FFF7A8FA04000920D2E7C04694
:10719000D864FF1FD464FF1F70B50A4E0400337813
:1071A0000D00FF2B0DD0042004F0BEFB011E08D003
:1071B000D0230370CE3B45708370C470307804F0E8
:1071C000C3FC70BD7843FF1F70B5040006200D009E
:1071D00004F0AAFB011E0AD0D0230370CD3B8370BC
:1071E000054B44701B688580187804F0ADFC002CBA
:1071F00001D0FFF767FF70BDD864FF1FF8B5264FB9
:1072000006003B680D001124002B05D10522234BFD
:107210001B78134202D112242000F8BD204A10240A
:107220001268002AF8D01278002AF5D0DB0719D5A9
:107230002B789A1E012A1AD80C2004F055FD13242D
:1072400038600028E8D000230A2243702900067025
:10725000023004F009FBFFF75BFF041E0AD0FFF7C2
:1072600031FFD9E700F012FB0028E1D1E4E7002B61
:10727000E2D0D0E70B4B1B78032BCDD11D20FFF7BD
:107280002BFA094B18800028C6D0084B0421187827
:10729000074A04F0B1FCBFE7D864FF1FD564FF1FA5
:1072A000F464FF1FD464FF1FD264FF1F0065FF1F3B
:1072B00060EA0000F7B50193194B14001A78052312
:1072C00006000F0012201A4221D0012920D1154BAF
:1072D0001D68002D1BD002201F2C18D8002C02D0B6
:1072E000019B002B13D0104B1F221E706E1C00211F
:1072F000300004F079FA01992200300004F0B4FA69
:10730000310020002C70002F06D004F0EDFBFEBDF4
:10731000064B12201D68DCE704F026FAF7E7C046AA
:10732000D564FF1FF464FF1F7843FF1FF064FF1F45
:10733000F8B50F4E12243368002B17D01B780F3C82
:10734000834213D100250B4F0221387804F084FAD0
:10735000094B042138781D8004F07EFA074B280081
:107360001D8033685C7004F01FFB04002000F8BD32
:10737000D864FF1F0065FF1FEC64FF1FD264FF1F6E
:1073800070B5012823D11B4C2388002B03D01A4A47
:107390001578002D07D0194B1B68002B02D01878E8
:1073A000FFF7C6FF70BD3B2B02D93C3B2380F9E7BA
:1073B000134E0221307804F04FFAFA22238892000B
:1073C00002215A43307804F0F7FC2580EAE70B4BA2
:1073D0001B68002BE6D00B4B1B785B07E2D5084BF4
:1073E0000221187804F038FA0022024B1A80FFF7C5
:1073F00069FED7E7EC64FF1FD064FF1FD864FF1F4E
:107400000065FF1FD564FF1FF8B51E4D28680028D2
:1074100003D004F049FB00232B601B4E306800288A
:1074200003D004F041FB00233360184F05243B7860
:1074300018002040234221D0154800F02BFA3B7859
:10744000234213D0202004F04FFC2860002813D0E2
:107450002022002104F0C8F9202004F045FC041E7D
:10746000306005D02022002104F0BEF9002004E0A5
:10747000286804F019FB2C601320F8BD00F00AFA0C
:10748000F4E7C046F464FF1FF064FF1FD564FF1FDC
:107490006C43FF1F10B50A4C23681A1E0ED000283B
:1074A00008D10130587004F07FFA002805D0236815
:1074B000002B02D00021FFF787FE0122100010BD33
:1074C000D864FF1FF7B5274E050033680191181ED9
:1074D00021D05C78244F012C30D1FFF7FFFD00282C
:1074E00025D02000FFF7F8F80400412814D91F4BDD
:1074F000022118781E4A04F07FFB1E4B3C3C1C8086
:10750000022233685A703B78002B14D1280001996D
:10751000FFF75AFE0120FEBDFA2292004243002AE4
:10752000EED0124B0221187804F046FCE8E7FFF792
:10753000D3F80200F3E700233B70EBE73B78002B26
:10754000E8D1032004F0F0F9011E08D0D023037025
:10755000CC3B457083703368187804F0F5FAFFF778
:10756000B1FDD7E7D864FF1FD064FF1F0065FF1F80
:1075700060EA0000EC64FF1F10B517498388020021
:107580008B4220D011D815498B4217D014490020C6
:107590005B1899B2012907D8926811785A42534171
:1075A000D8B2FFF7F9FD012010BD0E4A00209B184C
:1075B00007229BB29A424041C0B2F5E7836818782F
:1075C000FFF768FFF0E7836899785A78090218781E
:1075D0001143FFF777FFE7E70A20000006200000CD
:1075E000F8DFFFFFAFDFFFFF014B18707047C046A9
:1075F0007943FF1F10B5064C207001F041FA207846
:1076000004F0C2FA0521207800F062FD10BDC046EA
:107610000065FF1F0BB273B50D00002B00DBC4E04B
:10762000884B187804F0A8FB041E0ED00378912B29
:107630000FD0A22B00D1A1E0834B1878FF2852D0A5
:10764000210004F081FA00284DD18020000268401A
:1076500076BD43780F2B76D013D8052B70D00E2B28
:10766000EAD18088794B98422BD8794B98421BD825
:10767000784B9842E0D1A3681878591CFFF774F84A
:1076800038E03E2BD8D18378032B74D06CD8012BF3
:107690006ED0022BD0D1704B1B68002B23D05B68BF
:1076A000002B20D098471EE06C4BC0180C28C3D884
:1076B00004F0BAFA1DC2C2150BC20B0B0B3223C267
:1076C0003C00674BC0180728B6D8664B1B68002BD8
:1076D00009D01B68002B06D0200098470AE0A36859
:1076E0001878FFF7C7F8200004F00EFBADE7A0689C
:1076F000FFF762F800289FD0F5E7A3681B78002BFE
:10770000F1D0554B1B68002BEDD01B68002BEAD045
:10771000210055489847EDE74F4B1B68002BE2D0FE
:107720001B68002BDFD021005048F3E7504B1B684B
:10773000002BD8D05B68002BD5D021004348E9E767
:10774000FFF7EAF9CFE780884A4B984203D04A4BCB
:10775000984200D070E7464B1B68002BC3D05B6893
:10776000002BC0D02100D5E7153B012BBBD963E727
:10777000FFF798FAB7E7FFF77DFAB4E73F4B1B78BE
:10778000042B07D100236A4613800179408800F05A
:10779000C5FCA8E7364B1B68002BA4D05B68002B08
:1077A000A1D00100364898479DE7012421420AD024
:1077B000294B1B68002B04D05B68002B01D00020F4
:1077C0009847012043E78B070AD5264B1B68002BFF
:1077D00004D05B68002B01D020009847022036E7D8
:1077E0000421280008400D4200D131E7254E33889E
:1077F000002B21D0013B9BB23380002B1AD1FFF725
:10780000DBF800280AD0204B1C70164B1B68002B9D
:1078100004D05B68002B01D020009847FFF7C6F822
:10782000694601F001FD6846FEF7FEFF1D20FEF7E8
:1078300053FF308004200AE7024B187804F00CF85C
:10784000F8E7C0460065FF1F7943FF1F0E200000C8
:107850000120000009100000F864FF1FFEDFFFFF99
:10786000AFDFFFFFFC64FF1F0C2000000B200000B7
:10787000E064FF1F0D20000013200000D564FF1FEF
:10788000FFFF0000D264FF1FD064FF1F10B501F09E
:107890009BF910BD014B18607047C046FC64FF1F88
:1078A0000B880020162B01D817230420014A1380CF
:1078B0007047C046AA64FF1F00207047074A0300B4
:1078C0001188814207D091880020994202D101306D
:1078D0008000101870470020FAE7C0460865FF1FB7
:1078E000F0B58F7806000D00C5B01E2F15D1FFF73B
:1078F000E5FF051E03D10024200045B0F0BD0022A5
:107900003B003100C078009200F0B2FB0400A81CDC
:1079100000F0D2FBFF23EB70EEE7264B0624039327
:107920001B78FF2BE8D0182FE6D87B08224A013BB2
:10793000DB0002929A589446002ADDD0029AD318AE
:107940005B68002BD8D00878002802D14B78012B37
:1079500002D10624122FCFD107AFAB8869780097E8
:107960006446AA68A047041EC6D1AB78029A5B0899
:10797000013BDB00D318390030005B689847041ED8
:107980000BD1AB78042BB6D0039A310010782200CB
:10799000009700F06DFB0400AEE76A78002AABD1D7
:1079A000AA7805A93B88087130000A704B80FEF761
:1079B00047FBA0E77C43FF1F9CBF00111D4B37B561
:1079C000050098420BD000290AD1FFF777FF002865
:1079D00005D11948FFF772FF002800D0058037BD98
:1079E00001291AD1FFF76AFF041EF8D001235B4278
:1079F0000380A378FF2BF2D0FE2B07D00023E07882
:107A00001422009329001E3300F032FBA01C00F06A
:107A100053FB01235B426380E1E70229DFD1013997
:107A200001F0BEF80028DAD12800FFF747FF041E56
:107A3000DFD1D4E7FEFF0000FFFF0000022210B5F7
:107A4000074B52421A80074801325A809A80DA80E6
:107A500000F07EFA044801F025F8002010BDC04671
:107A60000865FF1FE1780011BD7900110388F7B5A3
:107A70000400002B02D102252800FEBD426802212D
:107A8000137825485268FEF7A5FD00282ED0234F15
:107A900001253A88002AEFD0802321885B02012546
:107AA0009B1A9942E8DC0C2004F01EF9061E31D026
:107AB0003B8822889C4600231800019561469DB2B0
:107AC000491989B2AA421BD8002801D062443A80E1
:107AD00000233000082208C0210003F0C5FE104A30
:107AE0001368002B13D100251660C5E762680221D8
:107AF00013780C485268FEF76DFD0028C7D1BAE72D
:107B000060681D014019418101330198D6E71A00D0
:107B10001B68E6E71325AFE70AC000117A43FF1F91
:107B20000465FF1F08C00011014B18707047C04664
:107B30007C43FF1F14230A0010B51A40194204D0D9
:107B40000122102101F048F810BD4B06F9D40120A4
:107B500088434000F8E710B514008B0604D50122D5
:107B6000102101F039F810BD08230A001A4019420B
:107B700002D14BB2002B0FDA102101F02DF80028B2
:107B800008D02300F2331B78002BECD0F13423789B
:107B9000012BE8D10020E6E703208907FAD4E2E7C9
:107BA000F0B51F00184B85B01C680190029103923C
:107BB000002C27D1200005B0F0BDA5683301ED18D9
:107BC0006B89019A934211D3029A93420ED8002FE7
:107BD00004D10A9B002B10D12C00EBE73B00297845
:107BE000039A6868FEF7F6FC0028F2D10136B6B2B7
:107BF000A388B342E1D82468DAE7A3680A9A5B89CC
:107C00001380E9E70026F3E70465FF1F37B50C0092
:107C10000A8849880123914217D3002A15D0651D8F
:107C200023792A0002210A48FEF7D4FC10230028F9
:107C30000BD023796188208800242A000094FFF764
:107C4000AFFF0A23A04200D0230018003EBDC0466B
:107C50000AC0001113B50A00088849880123884228
:107C60000BD8002809D00024137905320094FFF7BF
:107C700097FF0A23A04200D02300180016BD13B5B9
:107C80000A0008884988012388420BD8002809D0B7
:107C90000024137905320094FFF782FF0A23A042E3
:107CA00000D02300180016BDF0B58BB003904A88B1
:107CB00008880E000123824255D3002853D00023A8
:107CC000012704AC23700022718813000092FFF793
:107CD00067FF051E3ED02078002835D12B78022B77
:107CE00018D167706A8983000130E31880005A80D8
:107CF00069680222201803F0B7FD23780133DBB254
:107D00002370042B19D93B006889013080B2002B05
:107D1000D9D01FE002236370122358436A892318C5
:107D200004305A8069681022201803F09DFD2378E2
:107D30000133DBB22370002BE5D10C4A6B899B1811
:107D40005A425341DBB2DFE76378012BE4D12B7851
:107D5000022BC7D022780A23002A04D021000398DE
:107D6000FEF798F9002318000BB0F0BD0100FFFFEB
:107D70000F4BF0B504001868002816D083685D89A1
:107D8000A54207D88288AE18B44203DA12019A18C5
:107D9000934201D10068EFE71E005F891036A742C9
:107DA00004D1002900D00D801800F0BD3300EFE7AA
:107DB0000465FF1F70B505000C0008880021FFF75F
:107DC000D7FF03000120002B04D022002800197ADD
:107DD000FFF7C1FE70BDF7B50C0000250190230030
:107DE000EE331B78AB4201D800200AE06B00E65A64
:107DF00000213000E718FFF7BBFF002802D12680E2
:107E00000130FEBD017A0198FFF794FE002802D0F0
:107E10003B882380F5E70135EDB2E0E710B50400BB
:107E200008880021FFF7A4FF03000120002B03D0E6
:107E30002000197AFFF77EFE10BD0000054B1B687D
:107E4000002B01D1180004E09A6852898242F6D1D1
:107E5000988870470465FF1FF0B50E27002687B08D
:107E6000039302ABFF183E8005001F4B40891400AE
:107E7000984207D02B78013000976A6880B2FFF7EC
:107E80008FFE060002212B7818486A68FEF7A2FBD5
:107E900000280FD06C892000FFF7D0FF002802D007
:107EA000013C0419A4B2039B002B00D01C803000BD
:107EB00007B0F0BD02212B780D486A68FEF78AFBF7
:107EC0000028E7D102212B780A486A68FEF782FB76
:107ED000002807D0002EDED03B88A342DBD1748976
:107EE000013CDFE76C89DEE7FFFF00000AC00011FC
:107EF00008C0001106C0001110B50C00FFF7DEFC31
:107F000003000220002B0AD0002C00D023609B78B5
:107F10001720FE2B03D00138FF2B00D1002010BD0D
:107F200073B50D0001A904001600FFF7E5FF17283F
:107F300005D0002E04D129002000FEF727F976BDD8
:107F400001221021200000F047FE0028F3D0F6E7C0
:107F5000014B18607047C0461465FF1F37B56B466C
:107F60009D1D010004000222280003F075FE2B88ED
:107F7000B02B0ED12379122B09D12300FA331B78B1
:107F8000012B06D10121608800F0E0F801E01B2BF5
:107F9000F8D037BD10B5054B0421187000F098F8E3
:107FA000FFF74CFDFEF770FB10BDC0461865FF1FC4
:107FB0000020F0B50BB20F0087B0834234DA274BB4
:107FC000187803F0D9FE051E2BD00378A02B25D1FD
:107FD00003AE3100FEF7E4F8041E0BD1B378DB07E3
:107FE00024D51F4B06341B68002B03D03100688852
:107FF00098470400A868002801D003F03DFE002C3B
:1080000008D1184A039B1340174A934206D0B3780D
:108010001B2B03D00121688800F098F8280003F09A
:1080200073FE80200002784007B0F0BD0F4B1B6844
:10803000002B10D0310068889847041EDAD073787E
:10804000002BD7D1B27801A90A704B800C716888D7
:10805000FDF7F6FFCEE70624F1E7C0461865FF1FDF
:108060001065FF1F00FFFF00000112001465FF1FD5
:10807000F7B50190FC200D0017001E0003F054FC22
:1080800004001320002C12D0B02320002370089B82
:10809000F4226770658026710830002B08D0190023
:1080A00003F0E2FB2100019803F04EFD0020FEBD2D
:1080B000089903F099FBF5E710B5041E06D0007887
:1080C000FD2803D803F088FDFF23237010BD0000B6
:1080D0000A1F93B210B504000220032B05D882407A
:1080E0000020024BD1529B189C7010BD3865FF1FB9
:1080F0000B8870B5043B04000D000220032B0BD845
:108100000121200000F04CFD03001420002B03D0BF
:108110002900200000F0DEFB70BD000007B5130051
:10812000034A00920A00012100F02CFC0EBDC0465B
:108130005983001107B5019203220092024B0A00F5
:10814000122100F049FC0EBDD783001107B56B4624
:1081500001AA11800449D88008780633012802D189
:10816000190003F091FB07BD1965FF1F0C4B10B5FB
:1081700018700023FF210B4A138013819381938091
:10818000094A53801370517293819372D174D382D0
:108190001375517703F070FB00F0FCF910BDC04679
:1081A0004865FF1F3865FF1F1A65FF1FF0B58DB0CA
:1081B0006B46002003910C229B5E834200DBB0E003
:1081C0005D4B187803F0D8FD051E00D1A4E00378BC
:1081D000902B00D09DE006AF01004688380000F0EB
:1081E00013FA79680400002900D19CE03B88052B34
:1081F0006ED13B89032B1CD905AC200000F0A2F8FE
:108200006288172A61D83989131D994231D179685A
:10821000237804310291D90738D5607800F08EF9BF
:10822000071E06D0002303712378012B08D0132BDF
:1082300023D0A868002800D178E003F01DFD75E088
:108240006288029909A800F0A6F80290380000F0B0
:108250008BF909AA2378387A019200223100009222
:10826000029A00F012F9380000F064F9029B002B2A
:10827000DFD0300000F080F9DBE70378032BD8D1A2
:108280006288029909A800F0D6F8DEE7122B13D114
:10829000029909A800F0B5F8021EEAD127498B8897
:1082A000002BC6D0887909A92378019161780091C3
:1082B000310000F0EAF8BCE7002302AA9383300003
:1082C000617809AAFFF72AFFB3E71D4B0993F6E788
:1082D000042B02D09A1F012AABD8184A043B9B00FA
:1082E000995A0029A5D0D218907831003A0000F0B0
:1082F000AEF800289DD13B88042B03D0012130002B
:10830000FFF724FF012C04D1A868002801D003F056
:10831000B3FC280003F0F8FC8020039B00024340DC
:1083200018000DB0F0BD012800D182E70121300016
:10833000FFF70CFFEDE7C0464865FF1F3865FF1FDC
:10834000010017000B7803704B784370CB788A7864
:108350001B021343438070470A88030002700A8897
:10836000120A42700A88012A06D14A8882704A8815
:10837000120AC2700420704702208242FBD14A8850
:1083800004309A704A88120ADA708A881A718A88C8
:10839000120A5A71EFE710B50400012082420CD98D
:1083A0004B780A781B0213432380834206D1CB7893
:1083B0008A781B0213436380002010BD022BFBD17F
:1083C000CB788A781B02134363804B790A791B02AE
:1083D0001343A380F0E70B8803700B881B0A4370DC
:1083E0004B8883704B881B0AC3708B8803718B8802
:1083F0001B0A4371CB888371CB881B0AC371082089
:10840000704703000120082A14D14A780878120224
:1084100002431A80CA788878120202435A804A7945
:108420000879120202439A80CA79887912020243BB
:108430000020DA80704710B504000120022A05D11F
:1084400000204B780A781B021343238010BDF8B537
:10845000060010200F00150003F066FA040001204A
:10846000002C0ED0A0230C22290023806780201D21
:10847000002D07D003F0F8F92100300003F064FB71
:108480000020F8BD03F0B0F9F6E7F7B51E00009044
:1084900008AB142017001D78019103F045FA041E63
:1084A00012D0A2230370019B47704380099B057182
:1084B00046710C220830002B07D0190003F0D4F9C4
:1084C0002100009803F040FBF7BD099903F08CF9F7
:1084D000F6E737B5041E0FD04388002B0CD00025DB
:1084E000C1881323007A172201950095FFF7CDFF6D
:1084F000FF2365806372257037BD000010B50C49FD
:1085000004004A88002A09D08B89002B05D000205E
:10851000CB8A0222834201D010BD012213000A201F
:10852000434300204032C854C81842800472F3E725
:108530001A65FF1F0023438003707047094B002119
:108540001A0010B55C88002C06D01C79844203D137
:108550000A234B43D01810BD01310A330329F1D14E
:108560000020F8E71A65FF1F10B50400407A03F0F9
:1085700033FBFF23637210BD7047043010B580B227
:1085800003F0FAFA002803D00421494203F0B4FBB7
:1085900010BD000070B50025104CA0682580A58195
:1085A000A580A84202D003F067FBA56000250C4C13
:1085B0000C4B606D1D80230058331D70A84202D003
:1085C00003F05AFB656500256068002801D003F0C0
:1085D00053FB013508340A2DF6D170BDE065FF1F4D
:1085E0008465FF1FD465FF1F70B5041E09D1054DBA
:1085F0002880A881A880A868002802D003F03CFB4E
:10860000AC6070BDE065FF1FF0B54B8885B001938D
:10861000002343600A7905000F00022A00D07BE0A6
:10862000CA88032A17D98B685E7819783602DC78F5
:10863000D8790E4399781B7A24021B020C4303431A
:1086400053495BBA0B80331D93421ED1042C04D0D6
:10865000631F022B0ED9012015E0019A4D4B120128
:10866000D35A002B06D00198FFF7BEFF4A4A136980
:10867000013313610421B8682E812C80494203F034
:108680003BFB6860002005B0F0BD434D042C06D0D4
:10869000631F022B0FD9EB680133EB60DBE7019A14
:1086A0003C4B1201D35A002B05D00198FFF79CFFD9
:1086B0002B6901332B61374B30000293019B029AE7
:1086C0001B010193002301998C468B5213006344D4
:1086D0009C8003939E81FFF750FF039B041E9860CC
:1086E00016D00421B868494203F006FBFA8801005D
:1086F000043A200003F0B8F80199029AFB888A5ADC
:10870000043B9B18029A8B522B6801332B60A2E723
:10871000AB690133AB619EE71E4B0293019B1E01C7
:10872000029BF35A002B2DD002998C19A0680028C7
:1087300028D0012A26D1FA889B189BB27352A189AE
:10874000994217D39B1AC018B96803F08DF8029BA1
:10875000A289F35A934200D07DE700222B81A3889F
:108760002B80A3686B60029BF2520B4A5368013363
:10877000536070E7084A9368013393600198FFF7EC
:1087800033FF68E7044A536901335361F6E7C04693
:108790004A65FF1FE065FF1F5065FF1F70B5051E8E
:1087A00015D10B4C0B4B1880230058331870606D9B
:1087B000002802D003F060FA656525005035606836
:1087C000002801D003F058FA0834AC42F7D170BD4C
:1087D0008465FF1FD465FF1FF0B51700A12285B087
:1087E000920001934243394B06001B680C009B1812
:1087F000D933FF331D78FDF741FF0430854204DD96
:108800003000FDF73BFF0430C5B2BD4207D33A004C
:1088100000213000019B03F047F805B0F0BD2900AE
:10882000380003F0C9F92300C6B250331E70039319
:10883000019B29006365380003F066F8CBB2029310
:10884000002B02D0039B01361E70002623005033FC
:1088500003931B78B34204D8606D002831D1002007
:10886000DBE7029A2800002A04D0013B1000B34243
:1088700000D02800F700E719387003F085FA786017
:1088800000280ED03A78019902F0EEFF019A3B7869
:108890000136D3180E4A0193D369F6B20133D3617E
:1088A000D4E7039B18706065A74205D1084A1320DE
:1088B000D36A0133D362B0E7606803F0DDF90834AE
:1088C000F2E703F0D9F900236365C8E73409FF1F15
:1088D0005065FF1FF7B50D0007000421686803F01D
:1088E0000BFA2B89040003702B891B0A43702B8819
:1088F00083702B881B0AC3702E8902250436F6B2BA
:10890000F42E15D81B4B9F4214D10C2003F00CF809
:108910001135011E0CD0902303708E3B0371043B74
:108920004380154B8460C680187803F00DF900254C
:108930002800FEBD5C237B43104AD31800935833B4
:1089400001931B78002B0FD10300320038000099EF
:10895000FFF742FF019B05001B78002BE8D1380090
:10896000009903F089F8E3E7054A0725536A0133C4
:108970005362DDE7FEFF00004865FF1F8465FF1FAF
:108980005065FF1FF0B587B0009017200F0016004C
:108990000193FFF7F2FD1325041E19D00C98031E56
:1089A00002D00199201D9847030AE370052302AA0B
:1089B000A0700430908127700098667003A993809E
:1089C0000494FFF787FF051E02D0200003F054F93E
:1089D000280007B0F0BD0000F0B587B01F000CAB59
:1089E0001B780391059301210DAB06001C780492BE
:1089F00000F0D6F81425002821D02000FFF77EFDD6
:108A00000135041E1BD01149059B0A780370013201
:108A1000D2B2131EC68001D101231A000B7022713D
:108A20003000049B03990097FFF7ACFF051E09D1A6
:108A3000230021000648074A093302F0C5FE28003A
:108A400007B0F0BD002363802370F8E74C65FF1F7B
:108A5000D384001130750000F8B505000E00064CF7
:108A6000064F2368002B02D03100280098470434B9
:108A7000BC42F6D1F8BDC046F065FF1F0466FF1F7B
:108A80000123064A5B425380002313715362044A58
:108A9000136053609360D360136170470466FF1FD7
:108AA000F065FF1F0200002310B506499C0008591D
:108AB000002801D1625010BD0133052BF6D11320DF
:108AC000F9E7C046F065FF1F034A5388181A43426E
:108AD00058414042104070470466FF1FF0B585B012
:108AE00002930AAB1F780CAB1B88009008000E00A5
:108AF00001920393FFF7E8FF05001120002D1BD121
:108B00000E48FFF7E1FF04001520002C14D00622C8
:108B10000B99A771E01D02F0A7FE019B30002371A5
:108B2000029B29006371009B66802370039B656232
:108B3000E381FFF791FF280005B0F0BDFFFF0000C3
:108B400010B5FFF7C1FF04000220002C12D060888E
:108B50000121FFF781FF606A002801D002F0A4FF25
:108B600028220021200002F03FFE012300205B426A
:108B70006380207110BD000030B5074A074C55884E
:108B8000010013780020A54204D05B1A59424B41E2
:108B90005842104030BDC0460466FF1FFFFF000072
:108BA000084A10B501230C00904208D0FFF78CFF53
:108BB000031E04D0037923405A1E9341DBB21800F0
:108BC00010BDC046FEFF0000024B1879431E9841BD
:108BD000C0B270470466FF1F70B504000D00160098
:108BE000FFF772FF002804D10D4B9C4200D01430D7
:108BF00070BD416A03790520002907D012221A406E
:108C0000102A02D10520002EF2D10F20DB06EFD56D
:108C1000897E0C20A9428941494249420840E7E740
:108C2000FEFF0000030010B5002800D110BD03486E
:108C3000034A41889142F9D09847F7E70466FF1F3D
:108C4000FFFF0000002330B5C45CCD5C6C40D45401
:108C50000133102BF8D130BD0F23002210B5C45CB6
:108C600064002243CA54C25CD209013BF7D210BD52
:108C70000200010010B52032103102F0E5FE10BDF7
:108C8000F0B58BB00390102005931700049103F00A
:108C90002BF80090102003F027F8009B132401907C
:108CA000002B05D000280CD11324009802F0FCFE04
:108CB000019B002B02D0180002F0F6FE20000BB042
:108CC000F0BD102003F010F80600102003F00CF89F
:108CD00013240500002E00D1AEE0002819D0102288
:108CE000002102F081FD32002900039802F0ACFE61
:108CF000041E0ED133787F2B51D830000099FFF736
:108D0000ABFF009B1B787F2B53D801990098FFF78E
:108D1000A3FF300002F0C8FE002D02D0280002F0B0
:108D2000C3FE002CC1D1102002F0DEFF060010208F
:108D300002F0DAFF0290002E7CD0002878D03A00B2
:108D40000F3223000125121105D00F333B4015B21D
:108D50005A4253411BB26A1E1201002B33D0049BAE
:108D6000D2B298180099029AFFF76CFF013D1022C9
:108D70000021300002F038FDADB2049F2D017D19B5
:108D8000AF4242D0002C33D0300002F08DFE029B67
:108D9000002B00D189E7180002F086FE85E7290044
:108DA0003000FFF759FF28002549009AFFF74AFFD6
:108DB000A7E729000098FFF74FFF28002049019AF4
:108DC000FFF740FFA5E70F210F4004998A18D9B299
:108DD0008F4208D9D15C06A819540133102BF6D163
:108DE000029A0199C0E7791A48424141C901F2E764
:108DF0003900300006AAFFF725FF3200039806A9C4
:108E000002F022FE10370400BAE7002CBCD130007B
:108E1000029906AAFFF716FF320006A9039802F08E
:108E200013FE082204003100059802F01DFDABE797
:108E30001324A9E71324AAE7002800D06EE733E73C
:108E400010C00011F0B58BB00F0016000225009085
:108E500000283FD0002A3DD00B1DDBB21800029342
:108E600002F042FF1135041E34D0FDF747FD050026
:108E70003A000099201D02F0A7FDEBB20393E370C6
:108E80002B0CDBB22F0A00936370FFB22B0E237002
:108E9000A7700193FDF72CFD1022010006A802F037
:108EA00093FD2100029A04AB06A8FFF7E9FE051E18
:108EB0000DD1039B08223370009B04A9B370019B62
:108EC0007770F370301D02F07FFDFDF71DFD20006F
:108ED00002F0EAFD28000BB0F0BDF0B58FB00D0038
:108EE000149E039004920593002A03D102242000CB
:108EF0000FB0F0BD002EF9D00398FFF7E5FD142464
:108F0000071EF4D07278337812021A43B3781B0428
:108F10001343F27812061A43036A0192934201D373
:108F20000133E3D1002D03D03B7901249B07DED52B
:108F30000822002106A802F057FC059B13240433E5
:108F4000DBB21800029302F0CFFE051ECFD0059AC7
:108F50000499043002F038FD04223100280002F0A8
:108F600033FD3900102210310AA802F02DFD29002E
:108F7000029A06AB0AA8FFF783FE041E0FD108224F
:108F800006A908A802F020FD0822311D08A802F059
:108F9000A3FD012807D101990398FDF7C9FC28001A
:108FA00002F082FDA3E70124F9E7000070B51C4C34
:108FB00005002368181E10D0002D14D11A78002A3D
:108FC0000CD1981C083202F04FFC02F075FC013500
:108FD000002808D123681D70012070BD0A331800D5
:108FE000082202F041FC2368002BF5D0122002F089
:108FF0009BFC061E0DD0C123216803704570023111
:109000001022023002F030FC23683100587802F060
:109010009BFD206802F048FD00232360DCE7C0468A
:109020002C66FF1FF8B504002020FDF755FB0D4E00
:10903000A700BB590500002B0DD000280BD0D87815
:10904000FF2809D108492A000C55F3590748033372
:10905000611802F0B9FBF8BD290002F0C5FC002838
:10906000F0D1F8E74866FF1F3066FF1F7DA20011B0
:1090700070B5064D84006359002B05D0D87802F0F6
:10908000ABFDFF226359DA7070BDC0464866FF1F12
:1090900070B506008CB00C00150000213022684627
:1090A00002F0A2FB31001022684602F08DFC1D2068
:1090B00021000322684402F087FC6846FFF7D8FDD0
:1090C0002D21040003222800694402F07DFC2000C9
:1090D0000CB070BDF0B50700160097B001931CAB43
:1090E0001D7830221EAB00910AA800211C7802F0E6
:1090F0007BFB102239000AA802F066FC1022002136
:1091000002A802F071FB0722310002A802F05CFC09
:10911000072202AB9818631E9C41019902F054FC8F
:1091200002AB9C732B005A1E934102AAD3730021F9
:10913000102206A802F058FB06221D9907A802F08B
:1091400043FC1A2002ABC01806221F9902F03CFC17
:10915000102200990EA802F037FC102202AB0EA9D3
:1091600008781C78013A6040D2B2087001330131AE
:10917000002AF5D10AA8FFF77BFD102212A90400EE
:109180000EA802F071FB102206AB0EA908781D781C
:10919000013A6840D2B2087001330131002AF5D19A
:1091A0000AA8FFF765FD044310222098E4B212A933
:1091B00002F00AFC200017B0F0BD70B50E001400DC
:1091C0008CB00100102268461D0002F0FDFB31004A
:1091D000082204A802F0F8FB2100082206A802F0E9
:1091E000F3FB6846FFF744FD04001022280008A99D
:1091F00002F0EAFB20000CB070BDF8B506000D00CF
:1092000000243719AC4200D3F8BD02F095FD030AE3
:109210003B70631CDBB201379D4203D90234F0542A
:10922000E4B2EEE71C00EDE773B506000C00022582
:10923000002819D0002917D0032101A8FFF7DDFF6E
:109240006B469A793F231A40013313436A46300034
:10925000937101A92200FFF71BFF051E04D1032211
:10926000E01C01A902F000FB280076BD0378580736
:10927000DA08C00FD20080009B0710439B0F1843F1
:10928000C0B2704707230B40C908C9000B430370E5
:109290007047000070B50400FFF7EAFE134DA4000C
:1092A0006359002B21D0186A002801D002F0FCFB82
:1092B0002B59986E002801D002F0F6FB2B59D86E7E
:1092C000002801D002F0F0FB2B59186F002801D0C4
:1092D00002F0EAFB2B59586F002801D002F0E4FBA2
:1092E000285902F0E1FB00232B5170BD4866FF1F97
:1092F0000E4B8000C35870B50C00002B0FD09D683A
:10930000002D0CD02B78201D0B706B784B70A97C36
:10931000FFF7B8FF2B7E23726B69E36070BD1022EC
:109320000021200002F060FAF8E7C0464866FF1FFF
:10933000014B18607047C0464466FF1F074A030090
:109340008000825810B5002A06D0D088984203D1F8
:10935000012901D1FFF79EFF10BDC0464866FF1FDF
:10936000F0B5264E95B087000B93BB5905000991C7
:1093700012200A92002B31D0D888FFF7A5FB0400F9
:109380001420002C2AD0280010A9FFF7B1FFBB59E8
:109390001E781D6A002E23D00895FDF7EFFA07000E
:1093A0000020FDF7F1FA0790A379E61D069310ADB2
:1093B0000CA9089800F0E2FA0EA9280000F0D7FAEC
:1093C0000B9B0A990493069B09980293079B0396AB
:1093D000019300970EAB0CAAFFF77CFE15B0F0BD11
:1093E000FDF7CCFA06903000FDF7CEFAE31DA77921
:1093F000079310AB06000893DAE7C0464866FF1FE4
:1094000030B50C4C85002A59030085B00120002A94
:109410000ED018006946FFF76BFF2B591A78D888D1
:10942000054B002A00D1054B6A46072100F0D9FB05
:1094300005B030BD4866FF1F6F9900117D9900117E
:1094400030B5094C8500295985B010226846253170
:1094500002F00AFA2A591121044BD0886A4600F01A
:10946000C0FB05B030BDC0464866FF1F199A001109
:1094700030B5094C8500295985B010226846353130
:1094800002F0F2F92A591121044BD0886A4600F003
:10949000A8FB05B030BDC0464866FF1F579A0011B3
:1094A000F7B54D4F86001020F4590D0002F01CFC5A
:1094B000F3592062186A132200286CD0033A29005D
:1094C0009C6802F0D1F9F3591A780192002A58D118
:1094D0001E6A227D317B944651400122019F114238
:1094E00001D167461740217D914339432175377B70
:1094F0004F40BC4660460027800701D44F08174004
:10950000012102208F40227D82433A432275377B1E
:109510005740BC4660460027400701D497080F40DB
:109520000420227DBF0082433A432275627D0027DA
:1095300094466046727B42400A4201D167460F4022
:109540000121627D8A433A436275777B5740BC466E
:1095500060460027800701D457080F400220627D33
:109560007F00824317436775767B00227E40760733
:1095700001D4BA080A400426617D9200B1430A432F
:1095800062756A78002A08D06278002A05D0052220
:109590000533DA7700221000FEBD0422297911423A
:1095A00005D1A17C114202D10533033AF1E7019ABA
:1095B00021782C78002A02D10A00210014001822F8
:1095C0000429E8D8042CE6D805206043034A053373
:1095D0001218525CDDE7C0464866FF1F20C000112C
:1095E00010B50A001121024B00F0FBFA10BDC04675
:1095F000B39A00110B0030B587B001AD2B806B46DC
:1096000004001100981D082202F02EF92A000B21F7
:109610002000024B00F0E5FA07B030BDDB9A0011E4
:1096200010B50A001121024B00F0DBFA10BDC04654
:109630002F9B001113B50B0011006A4613706B4687
:1096400004000622581C02F00FF96A460821200087
:10965000014B00F0C6FA13BD4F9B001110B50A0074
:109660001121024B00F0BDFA10BDC0469F9B0011B6
:109670007FB505000B4BAA00D4580800002C0FD072
:10968000666F237FE28821780396266F0296E66E46
:109690000196A46E0094FDF709FC2800FFF7FAFD7F
:1096A0007FBDC0464866FF1F10B51721FFF7E0FFDA
:1096B00010BD000070B50A000D00064B0221040029
:1096C00000F08FFA060029782000FFF7D1FF300064
:1096D00070BDC0467F9A001170B586B000236A46FF
:1096E0001370836804001D78681E0A2859D801A9E0
:1096F00002F02AFB060633373B3F43474B4F5300EC
:10970000180000F042F9062312284BD000281BD184
:109710006088FFF7D9F90823002813D04279002A7E
:1097200047D1264B1A78072312070BD5244B1A680A
:109730000723002A06D01668002E03D0290001AAAC
:10974000B04703006A4613706B461B786088002B95
:109750002AD1FFF767FC06B070BD180000F06CF965
:10976000D4E7180000F087F9D0E7180000F093F96B
:10977000CCE7180000F0ADF9C8E7180000F0C3F915
:10978000C4E7180000F0F6F9C0E7180000F0F6F999
:10979000BCE7180000F013FAB8E7180000F013FA5D
:1097A000B4E707236A46137069466088FFF782FFB3
:1097B000D1E70523012AC5D1024BB8E7D564FF1FC5
:1097C0004066FF1F4466FF1FF8B52C4F8600F35913
:1097D00004000D00002B40D0DA8882423DD15A7837
:1097E000062A33D11A78002A2ED0012099681A6AE5
:1097F000097D014206D0157B054203D007225A702D
:109800000120F8BD0220014204D0157B054201D0A1
:109810000922F4E70420014204D0127B024201D065
:109820000B22ECE7164B1B68002BE9D05B68002B82
:10983000E6D020009847BB5900215B78122BDFD17E
:109840002000FFF715FFDBE70E4BECE7112A04D1F0
:10985000002900D032252900F2E7002D08D1200090
:10986000FFF732F9002803D0102302791343037164
:1098700021002800FDF798FAC2E7C0464866FF1F9E
:109880004066FF1F4466FF1F70B50E4E8500AB5942
:109890000400002B13D01B78002B11D10A4B1B683E
:1098A000002B04D05B68002B01D02000984773592F
:1098B0005B78122B03D100212000FFF7D9FE70BD89
:1098C000024BECE74866FF1F4466FF1F4066FF1F20
:1098D000094B8000C3581020002B0CD01A6A002AB4
:1098E00009D09B68002B06D0127A1B7E101C9A426E
:1098F00000D9181CC0B270474866FF1F70B503003E
:109900000D0014000220002A30D000292ED0137040
:109910000B78081D53704B789370FFF7A7FCE0702D
:10992000012002212B7A23716B7B034063716A7BD8
:109930000A401343042263716E7B16403343637104
:109940006E7BF608F600334363712B7B0340A371F3
:10995000287B014000200B43A371297B0A4013435D
:10996000A3712A7BD208D2001343A37170BD10B536
:109970000A0001000120FFF7C1FF10BD10B50A0069
:1099800001000220FFF7BAFF10BD70B506000C0001
:109990000220002E30D000292ED07378201D0B70AD
:1099A000B3784B70F178FFF76DFC012235792572A1
:1099B00071794B1008001340934010400343881006
:1099C00010408000C9080343C9000B436373B17999
:1099D0004B1008001340934010400343881002408E
:1099E0009200C9081343C9000B4321202373FCF7DD
:1099F00073FE854201D2122070BD2220257AFCF729
:109A00006BFE8542F7D823781820042BF4D86378AE
:109A1000012BF1D80020EFE7030010B50220002948
:109A200009D0002B07D00322481C0A7019000D3200
:109A300001F01AFF002010BD03000222080010B53B
:109A4000002B06D0002904D00E32591C01F00CFF67
:109A50000022100010BD030010B50220002909D01B
:109A6000002B07D00422481C0A7019000C3201F0A8
:109A7000FBFE002010BD10B5FFF7DEFF10BD030098
:109A80000220002906D0002B04D0052200200A70F5
:109A90001B784B70704703000220002B08D0002970
:109AA00006D05B7800200B70013B082B00D91830E2
:109AB0007047030010B50220002909D0002B07D001
:109AC0000622481C0A7019000A3201F0CDFE00205F
:109AD00010BD10B5FFF7B0FF10BD02000B00022053
:109AE00010B500290ED0002A0CD00721197011885A
:109AF00059701188090A997011180822D81C01F0B0
:109B0000B3FE002010BD03000A00022010B5002B98
:109B10000CD000290AD099785878090201431180A5
:109B2000901CD91C082201F09FFE002010BD0300EC
:109B300010B50220002909D0002B07D00822481CAC
:109B40000A701900921801F08FFE002010BD02006B
:109B50000B00022010B500290BD0002A09D00921E2
:109B60001970117818185970511C062201F07CFEEA
:109B7000002010BD10B5FFF75FFF10BD02000B0005
:109B8000022010B5002A09D0002907D05178197099
:109B900011180622581C01F067FE002010BD0300BA
:109BA00010B50220002909D0002B07D00A22481C3A
:109BB0000A701900063201F057FE002010BD10B5E2
:109BC000FFF73AFF10BD02000B00022010B5002A7B
:109BD00006D0002904D018005178FFF753FB00206D
:109BE00010BDF0B585B017001E006A4606230500BB
:109BF000080091819380FEF7C0FC1324011E02909F
:109C00000CD03800B047041E05D1280001A9FEF78A
:109C10006FFA041E02D0029802F02EF82800FFF717
:109C200001FA200005B0F0BDF0B504008BB0019141
:109C300015000021102202A801F0D6FD334EA70026
:109C4000B85900283CD0C388A34239D10378002BEF
:109C500036D14278062A18D102000100553235313A
:109C60000C3006ABFFF7A9FA002829D12000FFF736
:109C70002FFE020006A902A801F0F6FD200002A9AD
:109C800001F0BAFE01200BB0F0BD816E002917D0A3
:109C90000B8A112A28D19D420ED101981231093A1E
:109CA00001F01AFF012807D1BB5920009D6EFFF774
:109CB0000FFE29000200DEE732212000FFF7D8FC6A
:109CC0002000FEF701FF061E1BD0416A002918D0B4
:109CD0000B8AAB4215D108220198123101F0FCFE2B
:109CE00001280ED1716A0AE09D42E9D1082201984B
:109CF000123101F0F1FE0128E2D1BB59996E8A7E42
:109D0000B9E7200001F0D8FFBCE7C0464866FF1F56
:109D1000F0B56B4D87007E5985B033780290039380
:109D2000002B00D087E0B368346A0193707806286E
:109D300017D101221B7D134202D0217B114218D181
:109D40000222134202D0217B114251D1042213423C
:109D500003D0237B134200D08BE0019B5A7DEB594B
:109D600091E007380428F8D801F0EEFF032E42678F
:109D70008300B36E002B03D11C2001F0B5FFB06649
:109D8000EB599C6E002C1CD010220021200001F009
:109D90002BFD0298FFF79CFD01002000FFF72DFA34
:109DA00001F0CAFF2082200008211230FFF725FAB7
:109DB0000298FFF78DFDA076EB592100D888FFF7B8
:109DC0000FFC0822EB591CE0B36E002B05D01A00E3
:109DD000198AF0881232FFF70DFC0222019B197DCF
:109DE000EB5911423DD0207B10423AD0073208E0B7
:109DF000F488FCF7DBFD01002000FFF711FC0A22CC
:109E0000EB595A70029B9C002A595378073B042B4C
:109E100011D8D088FEF758FE00284ED0C3895A08C2
:109E2000D2182849029B0298CB542B59411804336D
:109E3000254801F0C9FC05B0F0BDFCF79FFD03000B
:109E40000120834201D100200393EB59DE88FCF707
:109E50009BFD039902003000FFF7ECFB019AEB59E0
:109E6000117D042211420CD0217B114209D00B221A
:109E7000C7E7F688FCF73CFD01003000FFF7EEFB7A
:109E80006BE7019A527D01210A4204D0607B0842AF
:109E900001D00C22B5E702210A4204D0607B0842BF
:109EA00001D00E22ADE704210A4204D0627B0A42AF
:109EB00001D01022A5E71222A3E7FA225200B0E750
:109EC0004866FF1F4C66FF1F87A2001110B5064BA6
:109ED0001A780423100018401A4200D00348FFF7F4
:109EE00027FA002010BDC046D564FF1F8043FF1F26
:109EF00070B50400FFF7D4FA051E43D12000FFF728
:109F00007FFA234EA400A0598268937CDB0708D512
:109F10000321036A1B790B40012B02D1017F0B4304
:109F20000377431DD97F8B1E022B0DD8022900D049
:109F30000121C088FCF790FF042133591A7F597022
:109F40000A431A77280070BD01290CD10223102280
:109F5000437000210C3001F047FC3059102135309E
:109F6000FFF74BF9EEE70529ECD10223D118437036
:109F700010220C3001F078FC04233259117F0B437E
:109F80001377EAE708251828DCD1053DDAE7C04653
:109F90004866FF1FF0B58BB0059143887E4F9E0049
:109FA000F45915000493002C15D1012902D000208A
:109FB0000BB0F0BD101D57781678FFF757F9EB6816
:109FC000320002932B7A0499019300903B00200009
:109FD000FCF70CFFEBE7E388049A934201D00820DA
:109FE000E6E72378012B00D1D4E0059B581E092811
:109FF00000D9CFE001F0A8FE05CE0A29CC506C852F
:10A000009AB229000498FFF773FFD1E720002900D6
:10A010001022453001F028FCB9594B78042B02D1AD
:10A02000013B4B70C3E70B000A00253335320C317E
:10A030000498FFF795F90498FFF702FA0522431EEA
:10A040009841BB59C0005A70B2E720002900102285
:10A05000553001F009FC049B4F4C9D002959049890
:10A060000A0006AB55320C31FFF77AF92959102254
:10A07000453106A801F030FD012808D10498FFF70A
:10A08000F7F90590002804D106222B595A7005983B
:10A090008EE708230593FAE763780C2B7AD1E36EF9
:10A0A000002B03D11C2001F01FFEE066BB59D86EC7
:10A0B00000286FD01022290001F0D6FBBB5904986C
:10A0C000DC6EFFF705FC0D22A076BB595A706EE7D7
:10A0D000E06E00285ED063780D2B5BD12B880822C0
:10A0E0000382A91C123001F0BFFBBB599A68517D55
:10A0F0000222114226D0186A407B104222D00C3234
:10A10000E4E763780E2B45D1236F002B03D1162093
:10A1100001F0EAFD2067BB59186F002803D0102218
:10A12000290001F0A1FB0F22BB59CFE763780F2B69
:10A1300030D1206F0622691C103001F095FBBB590D
:10A140009A68517D0422114203D0196A497B114259
:10A15000D5D100210498FFF78BFA28E7636F002B15
:10A160000DD0BB59586F0028F3D01022290001F000
:10A170007BFB0122BB5952425B6F1A61E9E7142055
:10A1800001F0B2FDBB5960675B6F002BE9D126E798
:10A190002978DFE707200BE74866FF1F10B5064C5C
:10A1A000207001F049FC06212078FDF791FF03485B
:10A1B000FEF778FC10BDC0465B66FF1F3D930011A3
:10A1C00000200BB270B50D00834216DA264B1878CA
:10A1D00001F0D2FD041E0DD00378922B0ED0A02BDF
:10A1E00037D0224B1878FF283AD0210001F0ACFC80
:10A1F000002835D180200002684070BD43780E2BC6
:10A200000BD03E2BEDD18378052B12D0082BE8D153
:10A2100081798088FFF7D8FA08E0154B82889A4246
:10A22000DFD183681878591CFEF7C0FE002817D1CB
:10A23000D7E7104B1B785B0712D50F4B1B68002B21
:10A240000ED09B68002B0BD0C289811D8088984757
:10A25000ECE7FFF741FAA068002801D001F00CFDFF
:10A26000200001F051FDC5E75B66FF1F7943FF1F2A
:10A2700018200000D564FF1F4466FF1F10B500784A
:10A28000FFF712FA10BD10B50078FFF7FDFA10BD08
:10A290000C234343084A10B59B185A68002A03D080
:10A2A000012901D1904710BD9B68002BFBD00029EC
:10A2B000F9D19847F7E7C0467866FF1F012383402E
:10A2C000094A10B5946B1C439463506B98435063D8
:10A2D000D46B20009843012901D120001843D0639A
:10A2E000116B0B43136310BD00800040F0B50024D8
:10A2F0000127154B85B0DA6B144E03921A6C01924C
:10A30000DA64019BE3403B4217D0039DE5403D40AA
:10A310000295E5B202992800FFF7BAFF316A736A25
:10A32000002908D03900002B01D00299794028007B
:10A33000FFF7C4FF01E0002BF9D101340C36172CD4
:10A34000DFD105B0F0BDC046008000405C66FF1F55
:10A35000064B01215A68C2400A4204D01B68C34020
:10A360001800084070471B6DF9E7C04600800040A8
:10A370000122064B8240002903D0D9680A43DA60E3
:10A380007047D9689143D960FAE7C0460038004069
:10A3900030B5032444430F4BE25C1B199C785D7875
:10A3A00001232D1B0135AB40013BA340A140DB4302
:10A3B0000C00122807D80849920052181168194059
:10A3C0002143116030BD054A11680B4023431360DF
:10A3D000F8E7C04667C0001108F0004014F00040E4
:10A3E000C21F70B5D4B20623092C0BD80125084C26
:10A3F0009540002908D00021FFF7CAFF23682B43AE
:10A4000023600023180070BD2368AB43F8E7C04603
:10A4100000380040214BF0B51B185B78022B21D18E
:10A42000032444431E4A1F4EA35C12199478012250
:10A4300015008540B76B013CE4B23D43A240B563D3
:10A44000194C122815D89B0000290CD117495B180C
:10A4500099680A439A600123205C154A8340116879
:10A460000B431360F0BD11495B18996891439960E3
:10A47000F1E70E4B00290DD159690A435A61225C5C
:10A480001328E8D00123203A93400A49086803437F
:10A490000B60E7E7596991435961F0E75C66FF1F7C
:10A4A00067C0001100800040ACC0001100F0004007
:10A4B000A0F00040A4F00040F8B500241B4E1C4D55
:10A4C0001C4B1B5D012B1FD1194A9269E2401A42B5
:10A4D0000BD00122B25693402200143AD2B2022A83
:10A4E00009D815494A6913434B61013402360C35CA
:10A4F000172CE5D1F8BD0022B2560F499200521830
:10A5000091680B439360F0E7022BEED1E7B238007D
:10A51000FFF71EFF01235840C1B23800FFF77AFF52
:10A520003800FFF715FF6877DFE7C04639C0001134
:10A530005C66FF1F5D66FF1F00F0004001220238CD
:10A540008240054B002903D059690A435A6170477C
:10A55000596991435961FAE700380040F8B50E0097
:10A5600001210F008740114A0400D368FD43BB431B
:10A57000D360831E8B4201D8FFF7E0FF002120004B
:10A58000FFF72EFF0A4A0B4B5168012E05D13943C4
:10A590001B1951605E700020F8BD294051600222F5
:10A5A0001C1962709A6915409D61F4E700380040FB
:10A5B000008000405C66FF1F012210B58240074BFF
:10A5C000002906D019680A431A600121FFF7C6FF67
:10A5D00010BD196891431960F7E7C046008000403C
:10A5E0000C2370B5002543430A4A29009B181D70AF
:10A5F000094B04001B185D70FFF7B0FF0123A34057
:10A60000064928000A681A430A6005490A689A43FD
:10A610000A6070BD7866FF1F5C66FF1F34800040D3
:10A620003080004070B504000E00FF2813D00325D1
:10A630000540FFF7D5FF084AA3089B009B183F225F
:10A64000ED00AA40AE4019682000914331431960E3
:10A650000121FFF78DFE70BD18380040F8B50C24BD
:10A660004443134B0500E4186368002B03D1A3682F
:10A670001220002B1AD0022201270E4B00215B1959
:10A680005A7028002770FFF769FF63681E1E08D004
:10A69000A3683E00002B04D02800FFF759FE464077
:10A6A000F6B228003100FFF709FE0020F8BDC046D1
:10A6B0007866FF1F5C66FF1FF7B5C420FF222B4B97
:10A6C00080001958002491433F3A0A431A508022CF
:10A6D000274F5202274E1A60274B1D5D002D21D0B7
:10A6E000A31E012B03D80121E0B2FFF727FF012DA4
:10A6F00018D11F4B9B69E3402B4213D0E3B21800E3
:10A700000193FFF725FE01000198FFF755FFE3B223
:10A71000143B022B1DD801217156184A8D405369F4
:10A72000AB4353613B7F002B0DD0E5B22800FFF710
:10A7300095FF2800FFF70CFE7B7F0100834202D0CB
:10A740002800FFF7A5FD01340C370236172CC3D1C2
:10A75000F7BD012100237156F3568D40074A9B0037
:10A760009B189A68AA439A60DCE7C04600E100E0C3
:10A770005C66FF1F39C000115D66FF1F00F00040DE
:10A7800010B501210400FFF7E9FE0123044A00206F
:10A7900011194B70A34091690B43936110BDC046E2
:10A7A0005C66FF1F70B50E0015000400FFF718FF70
:10A7B0000C236343094A20009B189D605E60FFF7ED
:10A7C0004DFFF021064B074A8900051E5A5002D062
:10A7D0002000FFF705FF280070BDC0467866FF1F08
:10A7E0000000FF1FEDA2001170B5134D07202C785B
:10A7F000002C1FD1982221005200280001F08CFA71
:10A800000123C420FF222B700C4B80001C635C636F
:10A810000B4B1C605C600B4B195891433F3A0A4349
:10A820001A50802252021A600D20074A074901F08F
:10A830009BF8200070BDC0465C66FF1F0080004092
:10A84000A0F0004000E100E0B9A60011B9A4001199
:10A85000030010B50620072B09D8054A137001F034
:10A86000A3FAD7210020034B034A89005A5010BD98
:10A87000A843FF1F0000FF1FC91BFF1F70B51D006D
:10A8800002240C2910D8094ACA40D2070CD5FBF77C
:10A890002FFF041E08D1059A04992800FBF744FFF6
:10A8A000FCF7B2FDFFF712FB200070BD1210000094
:10A8B00030B50D7802232C009C43184201D02B4365
:10A8C0001C0008252300AB43284201D02B00234362
:10A8D00020241D00A543204201D01C4325002A232B
:10A8E0000D70184204D011781E3B0B43137030BD1D
:10A8F0000028FCD10C2113788B43F7E7F8B51D0035
:10A9000006AB1B88140007AA0E000B201778002B3B
:10A9100027D10A78022A49D14A6850781178000272
:10A92000244A08438018042840D801F00DFA031285
:10A930001D1B2300F06801F0AFF8021CC0B2B84242
:10A9400000D93A1CD2B22000F1682A8000F08CFFB6
:10A9500006E00222F3681B882A8023701B0A6370BA
:10A960000020F8BD0622EEE701232B80F3681B7858
:10A970002370F5E7F368002B16D008222A801A8886
:10A9800022701A88120A62705A88A2705A88120AB3
:10A99000E2709A8822719A88120A6271DA88A2712A
:10A9A000DB881B0AE371DBE72B80D9E701202B80D2
:10A9B000D7E7C04600D6FFFFF7B516000A781D009E
:10A9C00008AB1F880C000123022A18D14A6850786E
:10A9D000117800022B4A0843801803280FD801F091
:10A9E000B3F902254439E06801F056F8C0B20723F4
:10A9F000B84204D37B190193152B02DD0D231800F7
:10AA0000FEBDE0682A003100C01900F02DFF6B4642
:10AA100000209B88E268D0541B4B1B68834203D004
:10AA20001B68834200D098470023E8E70B23002FE0
:10AA3000E5D1022DE2D1737832781B021343E2682C
:10AA40001380114B1B68002BEED01B68002BEBD042
:10AA50000120E8E70B23002FD1D1062DCED12A000B
:10AA60003100E06800F000FFDEE70B23002FC6D1C5
:10AA7000012DC3D132787533012AC0D8E3681A702A
:10AA8000D2E7C04600D6FFFF6868FF1F70B50C0014
:10AA90001500072837D801F057F9041436361B364D
:10AAA000242E182015290BD8184E1622002130000C
:10AAB00000F09AFE22002900300000F0D5FE0020B0
:10AAC00070BD18200229FBD11288114B1A80F6E7BD
:10AAD00018200829F4D10A000E48290001F0BCF81A
:10AAE000EDE718200129EBD10B4B10780B49DA69FF
:10AAF000FFF7DEFEE3E718200129E1D1064B1078CD
:10AB00000749DA6BF4E70220DAE7C0465068FF1F16
:10AB10002644FF1F1C44FF1FAC43FF1FD443FF1FED
:10AB2000F443FF1F030010B50020DB0704D5072105
:10AB3000024A034800F08CF810BDC046C4C00011A2
:10AB4000AC43FF1F054A03001068002803D0828829
:10AB50009A4201D1806870470068F6E7606AFF1F7B
:10AB60000A88030008009A4204D08A8804309A4276
:10AB700000D0002070470000F8B5F22200230D4FEE
:10AB80000D4E7968050042433370994200D07B60D6
:10AB90000A4C0021200000F027FE00231A007C60F0
:10ABA000AB4202D100203370F8BD01332280DBB20A
:10ABB000F234F5E7586BFF1F566BFF1F646AFF1FE7
:10ABC00073B56B4601900600684615001980FCF7C6
:10ABD0004DFF041E11D1002D0FD07689002E11D00B
:10ABE0000C2001F081F800280ED0084A0460136898
:10ABF00086808560002B02D11060200076BD1A008F
:10AC00001B68F7E70224F8E71324F6E7606AFF1FE2
:10AC1000012100220A4B10B549420A4C1980998043
:10AC20009A719A70084B2070012019805A60FFF7C2
:10AC3000A3FF2078FCF778FF0448FDF733FF10BD31
:10AC40007068FF1F606BFF1F586BFF1FFDAC00118A
:10AC5000022310B5002802D0FFF7B2FF030018004E
:10AC600010BD0000030010B50020DB0704D504214F
:10AC7000024A0348FFF7A4FF10BDC046D8C0001128
:10AC80002C44FF1FF0B50E2687B003930CAB1F8832
:10AC900002ABF6180500080031000292FDF768F8D3
:10ACA00004000120002C0FD03088FFF74BFF030079
:10ACB0000E20002B08D05E68002E05D02100280051
:10ACC000039B029A0097B04707B0F0BD0A4B10B53E
:10ACD000984207D10122002352420A808B708A8059
:10ACE0008B7110BDFFF73CFF0028FAD001235B42B7
:10ACF000038000238370F4E7FFFF0000F8B5050030
:10AD000001290AD1134E00243388F227AB4219D00F
:10AD100028001149FFF7DAFF06E0022904D10139C2
:10AD2000FDF73EFF0028EDD0F8BD3B00634372689D
:10AD3000D018D35A002B09D03A00002100F054FD5E
:10AD40000134E4B2054B1B78A342EED801235B42E9
:10AD50003380DDE7586BFF1F7068FF1F566BFF1FC6
:10AD600010B5FFF7FDFE03000020834200D0987865
:10AD700010BD0000F0B589B01C000EAB80CB039075
:10AD80001E8810AB1B78049202930B7A0D00DB0631
:10AD900016D42B780593022B24D00498FFF7D2FE0B
:10ADA000002812D003689C46002B0ED0029B220084
:10ADB000019329003B00644603980096A04705E0F4
:10ADC0000498FFF7BFFE002802D10E2009B0F0BDA5
:10ADD0008368002BF9D00A2229000398984700289D
:10ADE000D7D0F3E76B6858781A786B4B00021043A2
:10ADF0009842D2D8043B984210D2684B984242D035
:10AE000015D8674BC0180128C7D80B20002EDDD1FC
:10AE1000EB681A7859683A80200028E0614BC01826
:10AE2000032800D979E000F08FFF846A789E5E4B9A
:10AE30009842B2D10B20002EC8D101233B80EB6891
:10AE400031001B7823706889013080B2FCF790FFD5
:10AE50003A88031E0ED0017802328A183A8042895D
:10AE600062704289120AA27059680278E01C00F0F0
:10AE7000FBFC06E004323A8031000422601C00F042
:10AE8000B3FC0020A2E70B20002E9FD1EB6807A99E
:10AE90001E8804233B80330A300026706370FCF761
:10AEA00067FF051E28D004AB9A890E2304A95B18FE
:10AEB0003E49C668FCF7D0FF00280BD12B783C48F0
:10AEC0006A680599FBF786FB002803D1012304AAD1
:10AED0005B42D3813278022A06D17168201D00F0CE
:10AEE000C3FC3B8802333B800E2304AA9B181B88BB
:10AEF000A3701B0AE370C4E704ABDE81F4E70B2008
:10AF0000002E00D062E7E9680398FFF729FF0223CB
:10AF10003B802070000A6070B3E70B20002E00D049
:10AF200054E70222EB681B883A8023701B0A637087
:10AF3000A7E7E86800F0B0FDC2B203000720B24204
:10AF400000D243E70DD00299DBB27118994202DBBF
:10AF5000921BD3B20293029BE9681A003B808919C5
:10AF60005AE70023F6E70B20002E00D02EE7072239
:10AF7000EB683A801A7822705A7862705A88A27008
:10AF80005A88120AE2701A792271DA886271DB88B3
:10AF90001B0AA37175E7C0460429000002280000BF
:10AFA00000D8FFFFFFD6FFFF03280000FFFF0000CF
:10AFB00008C00011F0B58DB06B460020089120222A
:10AFC0009B5E83423DDAA64B187800F0D5FE071E43
:10AFD00032D00378B02B2CD10079023816281FD834
:10AFE00000F002FE17001E001E001E0031001E00B1
:10AFF00096001E001D011E0052011E0073011E005E
:10B00000CD011E0050021E001E001E008E021E00FA
:10B01000E302944B94491B8878880B80FBF71AF85D
:10B020003800FCF79BFF914B1B68002B01D03800C8
:10B030009847380000F068FE8020089B00024340DB
:10B0400018000DB0F0BDEE220021874800F0CCFBC7
:10B050000BAA3B7B7989388900923A000D32FCF7C4
:10B060009FFD0400804B1B78002C3FD146E0804BB5
:10B07000788805937F4B4100CB5A0BAE073BDBB280
:10B0800032880293002301937B4B210006930093A7
:10B09000059BFFF76FFE744D002810D1069B3A8A7E
:10B0A0001B889A420BD138000599123000F014FD2C
:10B0B000002804D02B7862899B00EB185A80162355
:10B0C00006A81B18328820007989FCF7C5FE2B786A
:10B0D00004009A00AA1851880029C3D00133DBB2BA
:10B0E0002B70002807D006A9C98A9180634A12886C
:10B0F0009A42BCD802E0012149429180002B04D041
:10B1000059497888FAF7DAFF8AE73E890A2479E014
:10B1100000253E89574B06937B88069A5B009B5A15
:10B12000033B9D4202DB002DF0D05BE0162206A817
:10B1300012183B7B798900923A0030000D32FCF7FF
:10B140002FFD0590002858D04689017A7888FCF7B1
:10B15000F1FC041E44D1464B78880793069B4100BE
:10B16000C95A454B0439C9B206AAD28A069302913C
:10B17000019400930599079BFFF7FCFD041E2FD156
:10B18000069B39491A88931C002D26D14B8079885B
:10B19000384B4900CB5A5119033B8B4220DD059BAC
:10B1A00031485B8941190B71A91C0135C9B2EDB257
:10B1B000059145191B0A2B71059B2D49043318185D
:10B1C00000F052FB2C4B059A1B88D318DDB22C4B98
:10B1D0009E4205D00136B6B29CE749889942D6D046
:10B1E000002D0CD0204C2800618800F01DFB207041
:10B1F00021007888FAF772FF12E7059CF0E7002C2F
:10B2000000D183E77B78142B00D109E716493B79FD
:10B210004E800B700C717888FAF712FF00E7162445
:10B2200006ABE41821003889FCF7A2FD011E00D10D
:10B23000B7E1788822880F4C45002C5B0A4D013C11
:10B24000E4B2029400240F4B01940095FFF792FDA5
:10B25000041E00D014E129007888FAF74FFFDFE6DA
:10B26000606BFF1F1843FF1F7868FF1F6C68FF1F8C
:10B270006C69FF1FA864FF1F5C6AFF1F1643FF1F56
:10B28000FFFF00007A68FF1F162406ABE4182100B8
:10B290003889FCF76DFD011E00D182E17888228893
:10B2A000AE4C45002C5BAE4D013CE4B202947C896F
:10B2B000AC4B01940095FFF75DFD041E00D0DFE06C
:10B2C00029007888FAF724FFAAE60025A44B1D8000
:10B2D0003B00F6331B78A24A78880792AB4208D924
:10B2E0009E4B12880693069943005B5A013B9A4293
:10B2F00003DB0799FAF716FF92E616246B00FB189A
:10B30000059306ABE418059B21001889FCF730FD76
:10B31000011E03D1059B01241E8973E77888924B97
:10B320002288069C099343001B5B904E013BDBB2D5
:10B330000293002300960193099BFFF71BFD041E57
:10B3400002D0059B1E895DE77B88069A5B009B5AAD
:10B35000079A108832881218934202DC1B1A013BAC
:10B3600033807F4C023032880999001900F07CFA52
:10B370002388328801359B182380EDB2A8E70BAAF9
:10B380003B7B7989388900923A000D32FCF708FC42
:10B3900000250590059B002B04D10A24002D00D127
:10B3A0006EE060E0059B7888197AFCF7C3FB01002A
:10B3B000041E63D1694C6C4B788806940993069BF4
:10B3C0004400E45A694B063CE4B20BAE3288079362
:10B3D0000294019100930599099BFFF7CBFC041E91
:10B3E0004CD1079B5E491B881A1D002D30D14A8025
:10B3F000059B5B4C5A8963191A716B1C9BB2E3184D
:10B40000120A1A71162306A832881B187989059822
:10B41000FCF722FDFF21AA1C2E1D03350B00059011
:10B4200092B2B6B2ADB2002803D006ABDB8AD9B275
:10B430001B0AA218651911712B714C4D301D2A88F9
:10B440004949201800F010FA2B88F618B5B2A1E788
:10B450004988914207D17A8806995200525AEB18CE
:10B46000053A9A42C4DC3E4C2800618800F0A4FBF7
:10B47000207021007888FAF75FFED1E5002DF2D127
:10B480003E89BFE6162606ABF61831003889FCF770
:10B490006FFC3D000400FA3500282DD0037A9B068E
:10B4A0000CD400227B893989788800923A000C32CA
:10B4B000FFF7E8FB041E10D03E8915E03088FFF747
:10B4C00041FB00281AD08368002B17D021001222DC
:10B4D00078889847041EE4D0EEE72B78002B02D141
:10B4E0007888FAF739FE00262B78002B00D097E5F4
:10B4F000002C00D194E585E60124DDE70E24DBE78E
:10B50000162506ABED1829003889FCF731FC041E1E
:10B5100047D0037A9B0611D4154A7B88118899423B
:10B5200003D01448814207D11380134BF2261D78B3
:10B530000023D9B2A94221D30924A1E72888FFF723
:10B5400001FB00282FD08368002B2CD02100122271
:10B5500078889847041EDFD092E7C046A864FF1F92
:10B560007868FF1F7A68FF1F6C69FF1F5C6AFF1F06
:10B57000586BFF1FFFFF0000566BFF1F3100594340
:10B58000546801336018615A0029D2D13C00083454
:10B590002100F22200F068F921007888FAF7E4FD32
:10B5A0003EE501246CE70E246AE71D4B1A887B8870
:10B5B0009A4231D07888FAF7E1FD31E5F223059817
:10B5C00051684343CD18C95A00291FD03B7A012B3B
:10B5D0000BD16C88AB887888AA1D0094FFF752FBCA
:10B5E000041E02D000233B722E88F2220021280084
:10B5F00000F0FAF800232B80059B0133DBB20593A2
:10B60000084B05991B78064A8B42D7D801235B4229
:10B610001380002CCED0F5E5002634000596EFE728
:10B62000586BFF1F566BFF1F70B504000E0015000E
:10B63000FFF796FA031E08D131000548FFF790FA8C
:10B6400003001120002B02D01C8000209D7070BDD3
:10B65000FFFF0000F8B50B4F06003B780D0014000B
:10B66000FF2B0ED00A2000F05FF9011E09D0B12394
:10B670000380002346800371C5800481387800F080
:10B6800063FAF8BD6D44FF1FF7B50F0008A9060067
:10B69000088809A90B240988002821D10234022B2B
:10B6A0001ED1557813782D021D432B008B43019337
:10B6B0007334002B14D1FB68300019000093FFF79E
:10B6C0004FFB019C85420BD02A0030000099FFF708
:10B6D000ABFF041E04D12A0030007989FFF7BAFFBE
:10B6E0002000FEBDF0B50E7885B003900AA805884D
:10B6F0000120022E0DD14C682778647824023C4347
:10B70000054FBC4205D10398DBB201960095FFF7C7
:10B71000BBFF05B0F0BDC04602290000034B10B5C9
:10B720001B68002B00D09847FEE7C046646BFF1FE4
:10B7300007B501A8FFF7F2FF044A05480021121AD5
:10B7400000F0EAFAF8F798F8FEE7C046686BFF1FCA
:10B750007044FF1F0000000001B40248844601BC91
:10B76000604700BF350E000001B40248844601BCAA
:10B77000604700BF5522000001B40248844601BC66
:10B78000604700BF8D12000001B40248844601BC2E
:10B79000604700BFB54C010001B40248844601BCBB
:10B7A000604700BFC521000001B40248844601BCC7
:10B7B000604700BF713AFF1F01B40248844601BCD4
:10B7C000604700BFC94A010001B40248844601BC79
:10B7D000604700BFA946010001B40248844601BC8D
:10B7E000604700BF6DBC000001B40248844601BC44
:10B7F000604700BF154D010001B40248844601BCFA
:10B80000604700BFC130FF1F01B40248844601BC3D
:10B81000604700BF6571010001B40248844601BC65
:10B82000604700BF0124000001B40248844601BC07
:10B83000604700BF350E000001B40248844601BCD9
:10B84000604700BFC136FF1F01B40248844601BCF7
:10B85000604700BFEDA5000001B40248844601BC6A
:10B86000604700BFB352010001B40248844601BCE6
:10B87000604700BFE94C010001B40248844601BCA6
:10B88000604700BF7918000001B40248844601BC3B
:10B89000604700BFE117000001B40248844601BCC4
:10B8A000604700BF9DA9000001B40248844601BC66
:10B8B000604700BF0519FF1F01B40248844601BC60
:10B8C000604700BFD91B000001B40248844601BC98
:10B8D000604700BF4550000001B40248844601BCE7
:10B8E000604700BF193BFF1F01B40248844601BCFA
:10B8F000604700BFB14E000001B40248844601BC5D
:10B90000604700BFDD66010001B40248844601BC07
:10B91000604700BF090E000001B40248844601BC24
:10B92000604700BF4538FF1F01B40248844601BC90
:10B93000604700BF1D4D010001B40248844601BCB0
:10B94000604700BF056A000001B40248844601BC9C
:10B95000604700BFF919FF1F01B40248844601BCCB
:10B96000604700BF8552010001B40248844601BC13
:10B97000604700BF4931FF1F01B40248844601BC43
:10B98000604700BF851F000001B40248844601BC27
:10B99000604700BFED3AFF1F01B40248844601BC76
:10B9A000604700BF5125000001B40248844601BC35
:10B9B000604700BF691F000001B40248844601BC13
:10B9C000604700BF3939FF1F01B40248844601BCFB
:10B9D000604700BF4551010001B40248844601BCE4
:10B9E000604700BFC9A9000001B40248844601BCF9
:10B9F000604700BF5147010001B40248844601BCC2
:10BA0000604700BF311B000001B40248844601BCFE
:10BA1000604700BFF94C010001B40248844601BCF4
:10BA2000604700BF291C000001B40248844601BCE5
:10BA3000604700BF692EFF1F01B40248844601BC65
:10BA4000604700BFC926000001B40248844601BC1B
:10BA5000604700BFE548000001B40248844601BCCD
:10BA6000604700BFED4A010001B40248844601BCB2
:10BA7000604700BFC51D000001B40248844601BCF8
:10BA8000604700BF3119FF1F01B40248844601BC62
:10BA9000604700BF055E000001B40248844601BC57
:10BAA000604700BFDD52010001B40248844601BC7A
:10BAB000604700BF014C010001B40248844601BC4C
:10BAC000604700BF1D4B010001B40248844601BC21
:10BAD000604700BF3D18000001B40248844601BC25
:10BAE000604700BFCD4C010001B40248844601BC50
:10BAF000604700BF4D1F000001B40248844601BCEE
:10BB0000604700BF8539FF1F01B40248844601BC6D
:10BB1000604700BF2526000001B40248844601BCEE
:10BB2000604700BF2124000001B40248844601BCE4
:10BB3000604700BF9D36FF1F01B40248844601BC28
:10BB4000604700BFE932FF1F01B40248844601BCD0
:10BB5000604700BF594F010001B40248844601BC50
:10BB6000604700BF413BFF1F01B40248844601BC4F
:10BB7000604700BFA930FF1F01B40248844601BCE2
:10BB8000604700BFE928000001B40248844601BCB8
:10BB9000604700BF5D17000001B40248844601BC45
:10BBA000604700BFC56D010001B40248844601BC76
:10BBB000604700BF2146010001B40248844601BC31
:10BBC000604700BF090E000001B40248844601BC72
:10BBD000604700BF4D39FF1F01B40248844601BCD5
:10BBE000604700BF1147010001B40248844601BC10
:10BBF000604700BF853BFF1F01B40248844601BC7B
:10BC0000604700BF5952010001B40248844601BC9C
:10BC1000604700BFF30E000001B40248844601BC37
:10BC2000604700BFA54F010001B40248844601BC33
:10BC3000604700BF5D3BFF1F01B40248844601BC62
:10BC4000604700BF456B010001B40248844601BC57
:10BC5000604700BF156B010001B40248844601BC77
:10BC6000604700BF810E000001B40248844601BC59
:10BC7000604700BF2933FF1F01B40248844601BC5E
:10BC8000604700BFD949010001B40248844601BCA5
:10BC9000604700BF3555000001B40248844601BC2E
:10BCA000604700BF053AFF1F01B40248844601BC4B
:10BCB000604700BFADAE000001B40248844601BC3D
:10BCC000604700BF091B000001B40248844601BC64
:10BCD000604700BF75A9000001B40248844601BC5A
:10BCE000604700BF0D52010001B40248844601BC08
:10BCF000604700BF3D4B010001B40248844601BCCF
:10BD0000604700BF5549010001B40248844601BCA8
:10BD1000604700BF434D010001B40248844601BCA6
:10BD2000604700BFB70E000001B40248844601BC62
:10BD3000604700BF9137FF1F01B40248844601BC31
:10BD4000604700BF2951010001B40248844601BC8C
:10BD5000604700BF713BFF1F01B40248844601BC2D
:10BD6000604700BF9136FF1F01B40248844601BC02
:10BD7000604700BFC539FF1F01B40248844601BCBB
:10BD8000604700BFF54E010001B40248844601BC83
:10BD9000604700BF017F000001B40248844601BC37
:10BDA000604700BF5934FF1F01B40248844601BCFC
:10BDB000604700BFC91BFF1F01B40248844601BC95
:08BDC000604700BF8B52010037
:10BDC800000101030202030304030502060207023D
:10BDD800080209030A030B030C020D000E030F03EC
:10BDE800100311031303140315001600493C001136
:10BDF8007D3C001100000000020000000ABE001196
:10BE0800192A0F180A000000F1590000FD2400004B
:10BE180041460100AD810011C1A100111576001144
:10BE2800B17F001165540011B5AF0011B150001178
:10BE3800593E0011893F001100000000161600004D
:10BE48000200000054BE0011F4FFF3FFD2FC000012
:10BE5800C94000110000000000000000547579611D
:10BE68000042322E30003030313500676974687511
:10BE7800622E636F6D2F70767678005448303500E7
:10BE8800020000009CBE0011292A282A272A262AF7
:10BE9800252A242A0A180000E20400007102000082
:10BEA80078EC000005000000744000001027000036
:10BEB80060F000000400000006640000204E00004E
:10BEC80000000000060000005C440000102700008D
:10BED8006CEE000007000000050000001F501D1058
:10BEE800023CB4000001150020000000A10200007F
:10BEF8003031323334353637383941424344454698
:10BF08000000000069580011BD5800110000000031
:10BF18000200000024BF00116F2A6E2A1A18EAD8FE
:10BF2800BC80F0FC60000000000000000000F3038B
:10BF3800B59747D6F613F7D777E6F0A7F47400005D
:10BF480001A00000000000006410B71DC8206E3B6F
:10BF5800AC30D9269041DC76F4516B6B5861B24D08
:10BF68003C7105502083B8ED44930FF0E8A3D6D672
:10BF78008CB361CBB0C2649BD4D2D38678E20AA0DA
:10BF88001CF2BDBDFB349B5F8000008000100000E8
:10BF98000000000017620011A17800113B62001137
:10BFA800A97C0011BF6200117F7C0011356300116C
:10BFB800557C0011876300111D7E0011EF6300118D
:10BFC8001D7E001121640011D77D00113563001119
:10BFD8000D7C0011AD630011B57D0011000000005B
:10BFE8000000000093640011B57D0011F564001194
:10BFF800B9780011052A042A012A002A02290328EF
:10C0080001280028011800180000000000000000A6
:10C018000000000000000087010102010201010286
:10C0280001020303040103010101010103030201E9
:10C0380003000D000E001000110013001401070189
:10C0480008010A010B011C011D0204020502070276
:10C05800080219021A021C021D0301030203170039
:10C068000201000504000807000B0A001716001D4E
:10C078001C010201010504010E0D01111001141328
:10C08800011716011A19020201020B0A020E0D020B
:10C098001110021413021716030504030807030BF3
:10C0A8000A030E0D0001020307090A0B0E0F1011F7
:10C0B80012141718191A1B1F20212200FDA800119D
:10C0C800B9A9001100000000020000000EC0001114
:10C0D80000000000E5B600110000000002000000AA
:04C0E8000CC0001177
:020000041FFFDC
:1000000000000000C13D001110BE00110CBE001127
:10001000A061FF1F000000000000000000000000C1
:1000200000000000000000000000000000000000D0
:1000300000000000000000000000000000000000C0
:1000400000000000000000000000000000000000B0
:1000500000000000000000000000000000000000A0
:100060000000000000000000000000000000000090
:100070000000000000000000000000000000000080
:100080000000000000000000000000000000000070
:100090000000000000000000000000000000000060
:1000A0000000000000000000000000000000000050
:1000B0000000000000000000000000000000000040
:1000C0000000000000000000000000000000000030
:1000D0000000000000000000000000000000000020
:1000E0000000000000000000000000000000000010
:1000F0000000000000000000000000000000000000
:1001000000000000000000000000000000000000EF
:1001100000000000000000000000000000000000DF
:1001200000000000000000000000000000000000CF
:1001300000000000000000000000000000000000BF
:1001400000000000000000000000000000000000AF
:10015000000000000000000000000000000000009F
:10016000000000000000000000000000000000008F
:10017000000000000000000000000000000000007F
:10018000000000000000000000000000000000006F
:100190004D33FF1F9531FF1FC166010000000000B5
:1001A000000000000000000000000000000000004F
:1001B000000000000000000000000000000000003F
:1001C000000000000000000000000000000000002F
:1001D000000000000000000000000000000000001F
:1001E000000000000000000000000000000000000F
:1001F00000000000000000000000000000000000FF
:1002000000000000000000000000000000000000EE
:1002100000000000000000000000000000000000DE
:1002200000000000000000000000000000000000CE
:1002300000000000000000000000000000000000BE
:1002400000000000000000000000000000000000AE
:10025000000000000000000000000000000000009E
:10026000000000000000000000000000000000008E
:10027000000000000000000000000000000000007E
:10028000000000000000000000000000000000006E
:10029000000000000000000000000000000000005E
:1002A000000000000000000000000000000000004E
:1002B000000000000000000000000000000000003E
:1002C000000000000000000000000000000000002E
:1002D000000000000000000000000000000000001E
:1002E000000000000000000000000000000000000E
:1002F00000000000000000000000000000000000FE
:1003000000000000000000000000000000000000ED
:1003100000000000000000000000000000000000DD
:1003200000000000000000000000000000000000CD
:1003300000000000000000000000000000000000BD
:1003400000000000000000000000000000000000AD
:10035000000000000000000000000000000000009D
:10036000000000000000000000000000000000008D
:1003700031B7001100000000000000000000000084
:10038000000000000000000000000000000000006D
:10039000000000000000000000000000000000005D
:1003A000000000000000000000000000491BFF1FCB
:1003B000000000000000000000000000000000003D
:1003C000000000000000000000000000000000002D
:1003D000000000000000000000000000000000001D
:1003E000000000000000000000000000000000000D
:1003F00000000000000000000000000000000000FD
:08183800706FFF1F4118FF1F34
:10184000024981F3088802F08FFB0000706FFF1FD0
:1018500070B500241E491F4A1F484C6308CA1B0567
:101860001B0DE4188242F9D11C4B80228B630021AE
:1018700009201B4B920519621A4B1B4DDA671B4B53
:10188000DA688243DA609A68194802409A60112047
:10189000296002F0B7F8112002F094F880226B6CF6
:1018A000112093436B64EE23DB006343114A1B0C4E
:1018B00013840122104B9A7201F022FC0F4B1B780B
:1018C000002B04D10E4B1021187802F065FA70BD80
:1018D000000005408805054000060540FF010000A6
:1018E00000F0004004E100E0003800403CF000401F
:1018F000FFDFFFFF7061FF1F2462FF1F5264FF1FA5
:101900005062FF1F10B502F067F9072804D01228B3
:1019100008D0022808D010BD044A0420136B0133FC
:101920001363F8E70220F6E71420F4E75065FF1F81
:10193000F8B507000C0026002500503630785135E8
:10194000002804D10300287058342370F8BD29788A
:10195000CA00481E8141A3183800A25C5B68C9B266
:10196000FFF7D0FF00280DD12B78DA00A218013341
:1019700050602B703378044A013B3370136A013393
:101980001362D8E70123DFE75065FF1F5C23434361
:10199000074910B5C9180B0058331B78012B05D126
:1019A000FFF7C6FF034A936A0133936210BDC04636
:1019B0008465FF1F5065FF1F10B502F02DF9064A20
:1019C0000121130010CB4942D967044B136002F088
:1019D00053FB200010BDC04600E100E010001000E5
:1019E00010B5040002F018F9024B1C6002F044FB31
:1019F00010BDC04600E100E010B5040002F00CF993
:101A00004021094A200013688B43136000F0F6FA66
:101A100001F07EFC0022054B01201A60044B0432C9
:101A20001A6002F0B1FAFEE71CF00040C4F000407A
:101A3000C0F00040431E5A425341A022F0B5D201EB
:101A40005B421340154D164A40019B182A18127E1E
:101A50008BB00191002A1BD01A000832D46F0022EB
:101A6000E6B206AFE4B294420EDC2818C369002B3C
:101A700008D0019902AA117106AA049202AA16734B
:101A800003A898470BB0F0BD1978B9540132EAE7C2
:101A90001A7D1A7806AB01261A70E6E71068FF1F58
:101AA00000400040F0B5254B04004001C25C85B009
:101AB000002A2BD01A18117E002927D0917E0029E8
:101AC00024D01179022921D11689D788D168F51B34
:101AD000ADB22A1C102D00D9102292B2BE4217D1ED
:101AE0001818012303710023C269C38003819A423D
:101AF00006D06846032103730171029301A8904741
:101B00000820002C00D0192001F0FAFA05B0F0BD31
:101B1000013C65426C41A0256442ED012C40084D1A
:101B20001B186419074D0633013A92B2AA42EDD050
:101B30001888461C1E80085C2070F5E71068FF1F9F
:101B400000400040FFFF00000F220E4B10B59868C8
:101B5000104002380A280BD802F00AF80D0A0B0AC6
:101B60000A110A0A0A0A060002210020FFF762FF92
:101B700010BD0121F9E70020FFF794FFF8E7DB6FC4
:101B8000F6E7C046004000400F220E4B10B59868A3
:101B9000104002380A280BD801F0EAFF0E0A0B0A9F
:101BA0000A120A0A0A0A060002210120FFF742FF70
:101BB00010BD01210800F9E70120FFF773FFF7E7E7
:101BC000DB6FF5E70090004013B5334C2378072B0B
:101BD0003DD8324B1A78324B002A39D1802219680D
:101BE00052020A431A60252001F0CCFE20232D4A20
:101BF00011680B43802113606B460422C9050868F5
:101C00000733104228D080210422C905C868104239
:101C10002ED080212020C905CA688243CA601422C0
:101C20001A701A78002A2FD18021C905C86820327D
:101C30000243CA6014221A701A78002A28D11A4B5B
:101C40001A7D22785A601D221A705932DA6013BD4B
:101C50001A6816490A40C5E7086802430A60142258
:101C60001A701A78002ACED01A78013AD2B2F7E761
:101C7000C8680243CA6014221A7019784A1ED2B288
:101C80001A700029F9D1C4E71A78013AD2B2C7E72D
:101C90001A78013AD2B2CEE7A843FF1F7044FF1F63
:101CA0003CF00040A043FF1F00200040FFFFFEFF6C
:101CB000564B70B51B68012B03D1554A936D013308
:101CC000936501F0D1FF534B534A1860534B544C6A
:101CD0001A600123534A1360534A13602378002B80
:101CE00006D006225149524802F0C6F8002323705C
:101CF000504A514B10681B78C1B2002B0ED14F4C8B
:101D0000C0B223785BB2002B4FDB237824785BB220
:101D100064B21B0424021B191B1813600B1C5029EE
:101D20004ED95023464A47491078DBB2FF22022899
:101D30004BD10868444C454D267890432A7896420A
:101D400054D9227824782E78023B5D10A31B6B4374
:101D50005201D31A10335B111843086002F024F9C2
:101D6000031F012B45D83A4B1B78002B06D0394B6B
:101D70001B78002B02D0002001F08EFFA122364BF1
:101D800092009978354B4A431B689B188322920036
:101D90009B181B78033B012B03D8AF20400001F0B8
:101DA000F3FF01222E4BDA8270BD237824785BB2D8
:101DB00064B2FF33FF341B0424021B190138ABE764
:101DC000CAB2022AAED20223ACE70868254C264DDF
:101DD000267890432A78964208D9227824782D785C
:101DE000023B5B10641B63435201B2E72378DBB212
:101DF000B2E70228D5D11D4B1B78013B022B03D93A
:101E00001B4B1B78022BCCD16C20C8E79809FF1F15
:101E1000FC0FFF1F9C64FF1FFF3F000014100340D6
:101E2000A064FF1F0C10034000100340D50BFF1FE0
:101E30007211FF1FB40003408C09FF1F680AFF1FC7
:101E4000490AFF1F94000340460AFF1F470AFF1F6D
:101E5000F908FF1F2209FF1F300DFF1F3409FF1F64
:101E6000BC0BFF1F440AFF1F450AFF1F1C09FF1F71
:101E70002309FF1F10B502F0E7F80022014B1A807A
:101E800010BDC0469864FF1F10B501F045FFA121A9
:101E9000054A89009478054A61431268044B521838
:101EA000528C1A8010BDC046300DFF1F3409FF1F31
:101EB0009864FF1F10B50D4B0D4A9978A1239B0024
:101EC0004B431268D218531DD97F0A4B1B88994285
:101ED00009D2441C07D0C82805D0D2695B1A5A43DE
:101EE000054B5343C01802F077F810BD300DFF1FAB
:101EF0003409FF1F9864FF1F7102000070B5244D64
:101F00002B68002B28D001F077FF2B68D8402B6876
:101F10000400002B27D001F077FF2B68D8401D4B21
:101F20001D4A9978A1239B004B431268D118D25CBB
:101F300091239B00002A20D0CA580132CA50174B67
:101F400017491B680868834214D3D23B181A012A28
:101F50001AD0144B186070BD01F04EFF124B196877
:101F600001F0A2FED3E701F04FFF0F4B196801F01B
:101F70009BFED4E70D495B18E8E7CA500C4B1B6881
:101F8000DB68E418201AE4E7F530FF30E1E7C046EB
:101F90001C08FF1F300DFF1F3409FF1F9C09FF1F86
:101FA0009C64FF1FA009FF1F1808FF1F2DFF3F00A3
:101FB000A464FF1F70B504000D00282916D103008A
:101FC000A433C2881B889B1A0B4A9BB293420DD93B
:101FD00006006A3605223100653001F0EDFD00286B
:101FE00004D13100200001F037FE70BD290020002F
:101FF00001F04AFFF9E7C046FE7F0000F8B5050092
:10200000012001F031FF134CA36AA26A9342FBD175
:10201000114E336001F0C8FD1049030008601048FC
:10202000426894460F4A17680022BC4501D24268B4
:10203000BA1A0D4802603268AD18A422E562606ADF
:10204000520302436262094A1278002A01D00F3B10
:102050000B60F8BD00F00040340AFF1FE408FF1FCA
:1020600028100040180AFF1F1C0AFF1F1C09FF1F31
:1020700070B580241025E405A3682B43A36002F00B
:102080000BF8A368AB43A36070BD0000F7B5160062
:1020900080221C001023D2050191916805000B439A
:1020A000936000225A4BD7301A6001F025FF9D2320
:1020B0002A002F009B00EB58CA3201210092FC3706
:1020C000002B01D00021009A386801F0D5FD2900CD
:1020D000009BCB311A784F4BD3351A604B780A7876
:1020E0001B0213438A7812041A43CB781B0613434E
:1020F000494A1BBA13604B790A791B0213438A7948
:1021000012041A43CB7931001B061343434A1BBA0E
:1021100013606B782A781B021343AA7812041A43BF
:10212000EB781B0613433E4A1BBA1360019A330235
:1021300013433C4A13603C4B22001B1B9C46032963
:102140003DDCB3089A0013005142B21A032A46D16B
:10215000354AE018511A827840781204000202438E
:10216000E05C043302430A600022FF2B4BDDF022C7
:102170002E4B12011A600F222D4B1A602D4A136844
:10218000002BFCD00023224A27491360091B321D73
:102190000B191B68043A180A23706070180C1B0E88
:1021A000A070E3700434002AF2DC802210213B6826
:1021B000D20501333B6093688B439360F7BD634660
:1021C000D578981893782D061B042B43157804397D
:1021D0002B43557804322D022B430360AFE7022ACC
:1021E0000AD1114AE05C511AE218527812020243F5
:1021F0000A6004339BB2B7E7012AB5D10A4A521AE2
:10220000E15C1160F5E7084959180A600433ACE74E
:10221000000004403C000440380004403400044006
:10222000300004400C00044000010440040004405D
:102230001000044014000440F7B5150080221C0073
:102240001023D2050091916807000B43936000238F
:10225000654AD730136001F04FFE9D233E009B007E
:10226000F9583B00CA363200FC33002900D07FE029
:10227000586801F001FD390032785C4BCB311A60AF
:102280004B780A781B0213438A78AC4612041A432F
:10229000CB78281D1B061343554A1BBA13604B7994
:1022A0000A791B0213438A7912041A43CB791B065D
:1022B0001343504A1BBA13604B7A0A7A1B0213432A
:1022C0008A7A12041A43CB7A21001B0613434A4A26
:1022D0001BBA1360009A2B021343484A1360220072
:1022E000474B1B1B0093009BCE785B1801938B78A8
:1022F00036061B0433430E78043833434E780431DA
:1023000036023343019E33600328ECDC0321A80826
:10231000431C9B002940800003292BD13849E51834
:102320005E18A9786D78E35C09042D0229431943EE
:102330003160030008330021FF2B2DDD314B324982
:1023400019600F21314B1960012327490B60304B75
:1023500019680029FCD006211B680B40042B20D0F3
:1023600080220020D20593680A318B439360FEBD22
:1023700001217DE7022908D121495D18E11849783A
:10238000E35C090219432960D3E70129D3D11C4931
:102390005918E35C0B60CCE7194818180160043346
:1023A000CAE7002310490B606346002B0CDC3B009E
:1023B000FC335A68102101325A608022D20593689A
:1023C00001208B439360D2E7009B9B181B68190A7E
:1023D00013705170190C1B0ED37004235B42917063
:1023E0009C440432E0E7C046000004403C00044046
:1023F0003800044034000440300004400C00044025
:102400000001044004000440080F000010000440D4
:102410001400044070B5061E19D002225A4B9B7955
:102420009343012B13D1594B1A78FF2A0FD15A78B5
:10243000FF2A0CD19A78FF2A09D1DA78FF2A06D12F
:102440001A79FF2A03D15B79FF2B00D199E0504B19
:102450000C201A78012A08D000224E4D1A702978D3
:102460000B00093B042B01D8212070BD4B1F012B11
:10247000FAD9454CA37B042B00D982E0A279032A28
:1024800000D97EE09A1ED2B2012A02D860881F28A5
:1024900077D9002E56D0012E73D1A0880128E3D021
:1024A000002907D1581E032803D801F061FB121739
:1024B00015122E702978481E032811D80025364B96
:1024C0001D602823237501F02FFDA84227D0A58089
:1024D000CAE702212970EDE70421FBE70321F9E7B0
:1024E00007390129C0D82D490968C96A8906BBD5B1
:1024F0002B4908780028B7D1012A01D9002BB3D184
:1025000002230B708021274D2633890128782375FB
:1025100001F01AFC80212878890101F03DFC01239B
:10252000A380214B1B78002B0AD0FA2280211F4B5D
:1025300092001B8809025A431A4B187801F05CFB81
:10254000002092E701F068FB2B78A680073B012B67
:1025500003D917482E7001F01FFD114B114C1A784A
:10256000002A06D080210022207889011A7001F00B
:10257000EBFB01F081FD80212078090201F0E4FBF2
:10258000DEE7122071E7C046A60BFF1F6B09FF1F95
:102590001A09FF1F1C09FF1F4809FF1FA464FF1F22
:1025A0002309FF1F1B09FF1F2109FF1F2C09FF1F04
:1025B0000010004010B5002901D001F0FDFB10BD56
:1025C000F7B5604B01919978A1239B004B435E4A7C
:1025D000060014681022E418D6235B00E058362366
:1025E000FF33E35C00279343222B41D1574B0F3A33
:1025F0001A600760012501F027FB019B1880E82382
:102600005B00E35C002B01D0B34258DD0023504F48
:10261000FB70AD33FF33E3581A68002A03D09B8860
:10262000DB439B071DD03823FF33E35C002B18D01E
:102630009B235B00E35C002B13D1D133FF33E35CBE
:10264000B3420EDAA4235B00E15AE018090A023112
:1026500001F0F2FB23000122FE33013E01351A870F
:10266000FA70E8235B00E35C002B2AD0A8B2FEBD21
:1026700003683D00002BBED081880430090A023176
:1026800001F0DAFBD6235B00E3581F60B2E72300BA
:10269000B133BA00FF339858013781880430090AF2
:1026A000023101F0C9FBE8235B00E35CBB42EEDCD6
:1026B000E822F61AED1800235200A354A6E70027DB
:1026C000F1E7200001F080FB00281FD0002E1DDD67
:1026D0007319882647190193B600200001F03CFBCE
:1026E0005A30800020184068013581880430090A7A
:1026F000023101F0A1FB200001F07EFCA35901335F
:10270000A351BD4202D0019B9D42E6D1114BE35C37
:10271000002BABD095239B00E35C002BA6D00E4B87
:10272000E15A0029A2D00D4AA35C994202D9013393
:10273000A3549BE700231A212000A35401F01CFCA2
:1027400094E7C046300DFF1F3409FF1F00140340FB
:10275000E010FF1F5A020000720200005E0200003B
:102760000D4970B54A6E0D4CD2038B69D20BA24253
:1027700006D80B4D0224AA4204D901F035FB70BDE6
:1027800002246442E21815007E2425402242F4D03F
:10279000A3432B438B61F0E700F000400A200000C8
:1027A000FC1C0000F8B51D4B1D4F1A78002A10D1F3
:1027B000BA7B002A02D101321A7003E0032AFAD050
:1027C000022AF8D001F0B0FB00220120154B1A704C
:1027D000F8BD154B154D1C68154B9E7801232B70C9
:1027E0002878C0B200F09EFBBB7B002B0BD101F020
:1027F000B3FBA1239B007343E41883239B00E418DD
:1028000023782B70E4E7032B02D101F00DFCF0E7F5
:102810000020022BDCD101F0AFFAEAE71C09FF1F10
:10282000A60BFF1F2309FF1F3409FF1F490AFF1FC3
:10283000300DFF1FF0B587B00EAD2F780FAD2D789E
:102840000593AC46634614000E4D0CAA12782E7800
:1028500003930D9B009201932200059B029701F0C8
:10286000F3FA2E70012C01D0042C08D180220649E5
:102870008B889343054A1278D20113438B8007B0AB
:10288000F0BDC0461C09FF1F6C11FF1F7809FF1F18
:102890000B001B3B70B504003020E02B0DD813005B
:1028A000E025493BFF3B9BB2ED00AB4205D8034B13
:1028B000200019825A8201F057FA70BD8410FF1F60
:1028C00010B501F0D1F9054B00205B68052B04D948
:1028D000034A5268D20200D4980810BD001000408C
:1028E000FCE100E070B501F097F90D4B1B68FC337B
:1028F000DC691D6AFFF7E4FF6419844204D2094BC6
:1029000001241B68002B07D004220024064B1A70F8
:10291000064A93690133936101F0AEFB200070BD5C
:10292000A464FF1F9809FF1F2309FF1FFC0FFF1F4F
:1029300070B50C4D2B68FC335C6A01F06DF9FFF744
:10294000BFFF2B680025FC339B6AE318834204D247
:10295000054B1B68AB4200D1051B01F08DFB280025
:1029600070BDC046A464FF1F9809FF1FD722044B07
:1029700092009B5810B5002B00D0984710BDC04660
:102980000000FF1F10B501F0DBF8FFF7EFFF27494C
:10299000274BCA6D274C1A4084235B001343CB6539
:1029A000254B1B68186A01F05FFA244B244A1A6011
:1029B000244B254A1A60A022244B52001A60244B53
:1029C000187801F021FB2000224901F075F900235D
:1029D000A3600233A360204B2049236003232048D7
:1029E000A36001F069F910221E4BFF201A608022BB
:1029F00052031A60802292031A60802212041A6025
:102A000001F04AF9012001F03FF9FA20400001F0FD
:102A100093F9582001F0B8F9134801F00DFB01209B
:102A200001F072F9072001F07FF910BD00F00040BD
:102A300000FEFEFF14100040A464FF1F00000340CE
:102A40000180063DBC00034034080000A4000340A0
:102A50004A0AFF1F71020000C3090000FFFF3F0088
:102A60002810004000E100E030750000674E336838
:102A700088331B6883F3088801F02EFA644A65499D
:102A8000136800200B401360634B644A1B68934239
:102A900000D1A6E001F090FA0221614A13688B434D
:102AA0001360FFF76FFF5F4B5F4C1878C0B201F007
:102AB0002BFA0023A3600233A3605C4B0120236048
:102AC00001F0D2F90323A36001F0C6F9040001F07C
:102AD000CBF8050001F0C0F9554B186001F00CF976
:102AE000544B1968621A531EA14200D2130080226F
:102AF000D203934201D39B029B0A3268D16AC90771
:102B000000D471E04C491C0C09689BB24C435943FA
:102B10002402090A641803264849FC3293680A68AB
:102B200047489B1A474A0768126847499B18474A13
:102B30009A1833409208DB190A600360042B03D90A
:102B4000013233400A6003600E684149A619300023
:102B500001F0AAF83F4F3E493B68C3183B60300084
:102B6000019301F031F83C4E306808183849306064
:102B7000884205D9019B01333B6001F025F83160A3
:102B800001F0A2F8354B1B78002B0DD001F06CF84A
:102B9000334B621B196812188A4232D24919091B39
:102BA000091A304801F088F82F4E337A002B0ED0E6
:102BB00001F05AF8621BF1681218914224D94919A0
:102BC000091B091A294801F077F800233372284BB2
:102BD00083F3088801F048FA002001F0EDF901F0D4
:102BE0006BF901F0E9F95CE7DC0199000234641A41
:102BF0005900641A09214B438033CB40A408E418E0
:102C000089E7FA218900CCE71A49DBE7A464FF1FB2
:102C10001CF00040FFFFC1FF0C0AFF1FB64121035B
:102C200010000040490AFF1F14100040C3090000B3
:102C3000100AFF1F340AFF1F380AFF1F200AFF1F58
:102C4000280AFF1F1C0AFF1F240AFF1FC4090000D7
:102C5000710200006008FF1F2C0AFF1F1C09FF1FE4
:102C6000E408FF1F00100040740BFF1F3C100040E1
:102C700000000020DC050000A022054B92009B58BC
:102C800010B5002B01D0984710BD01F0CDF8FBE73F
:102C90000000FF1FA122054B92009B5810B5002B8E
:102CA00001D0984710BD01F0BFF8FBE70000FF1FFF
:102CB000A222054B92009B5810B5002B01D09847DB
:102CC00010BD01F0B1F8FBE70000FF1FA322054B88
:102CD00092009B5810B5002B01D0984710BD01F011
:102CE000A3F8FBE70000FF1FA422054B92009B58AE
:102CF00010B5002B01D0984710BD01F095F8FBE707
:102D00000000FF1F70B500F0AFFF4F4B186001F0DF
:102D1000A3F90400C30702D400F0E6FF70BD00224F
:102D20004A4B1A604A4B18780138042829D800F019
:102D30001FFF0320181C2400200001F0C5F8012803
:102D4000ECD0444C2378042B6ED101F0A5F8002878
:102D5000E4D000F021FF582001F016F80223237080
:102D6000DCE7200001F030F9E9E7200001F08CF900
:102D7000E5E7200000F048FFE1E7200001F094F8CB
:102D8000DDE701F011F90500012808D1324B1B786D
:102D9000053B012B03D82000FFF76EFFD1E72D4B39
:102DA0001B78022B01D0052B20D1022D28D12B4BD3
:102DB0009B7BAB431CD12000FFF76CFF264B1878A0
:102DC0000128BED16405BCD4244925224B7B034293
:102DD00005D1233A13405A42534126331A000B7D42
:102DE0009342AED9322001F0A7F8AAE7022D07D10D
:102DF000194B1B78052B11D12000FFF759FFDDE798
:102E0000012D0BD1012B03D12000FFF75FFF98E7C5
:102E1000062B03D12000FFF767FF92E7200001F0A7
:102E200003F8022D8DD1C9E7032B04D10C4B987CFC
:102E300001F08AF872E7072B00D06FE7094B987B07
:102E400001F0D2F86AE7C0469C09FF1F9809FF1FEE
:102E50009009FF1F2309FF1F1C09FF1FA60BFF1F5F
:102E6000BC0BFF1FD40BFF1FFA210A4B0A4A490073
:102E70001A640A4A5A500A4A04395A50094A08310F
:102E80009A64094A5A50094A5C315A50084ADA662B
:102E90007047C0460000FF1F3528FF1F3129FF1F64
:102EA000E528FF1F1524FF1FA527FF1FB51EFF1FC5
:102EB000891EFF1FF7B50B0CFF270122009300238B
:102EC0003C001E001D009446019089B262469A4063
:102ED0001000084018413618B6B2FF2F02D1012E5B
:102EE00000D19FB2009802401A41AD18ADB2FF2C3C
:102EF00002D1012D00D19CB20133102BE6D1032069
:102F0000012E07D1012D04D1019B2401E4191C706D
:102F10000138FEBD102EFCD10238102DF9D0023040
:102F2000F7E700008023F7B59C46264B264F019318
:102F30002649274A274D284C284B02281AD160469B
:102F400038600868264E30408026360330430860DB
:102F500001990978002909D11660224A2A60224A7B
:102F60002260E02219689143A03A1BE08021C90247
:102F70001160F2E766463E600F68194E3E408027BA
:102F8000FF023E430E600199097800290DD11760B8
:102F900001280ED1154A2A60154A2260E0221968DC
:102FA0009143C03A0A431A60F7BD8021890211603B
:102FB000EEE7E0210F4A02432A600F4A22601A68B6
:102FC0008A43F0E74B0AFF1FE0000340D8000340AC
:102FD00090000340000003405000034040000340C5
:102FE000FFFFE3FF0280063D804508220180063D89
:102FF000806608220080069880550822F8B51E4B8E
:1030000080261A68002014003440324232D11A68F7
:103010001A4F32431A6001223B68063093433B60EB
:1030200000F022FF0122164D2B681E432E603B68E4
:103030000A2613433B608027BF00124B1B683B42AC
:1030400011D1013EF6B2FF2E09D17E220E4B1C6833
:103050002B68E40B1440934323432B6005E00820C6
:1030600000F002FFE9E7002EEFD180222B68600814
:1030700093432B60F8BDC046C4F000405CF00040B4
:1030800018F0004068F0004060F0004010B500F01B
:103090002BFF01215820034A00F0A6FDFFF7AEFFE9
:1030A00010BDC046600AFF1F10B5782200210348FA
:1030B00000F0B2FE00F090FE002010BD9867FF1FE8
:1030C00070B5040000F0A8FD00230C200B4A01009D
:1030D00059438D18515C00290DD0A14208D101231C
:1030E00000246B7000F0F8FD00F0C6FF200070BDFA
:1030F00001330A2BEBD11224F6E7C0469867FF1F75
:1031000070B5040000F088FD002319001D000D4A71
:103110001078002806D0A0420CD1557001310C3235
:103120000A29F5D1002B0AD100F056FE00F0A4FFC9
:10313000002070BD5078461EB0411B18EEE700F02D
:10314000CBFDF3E79867FF1FF7B504000C200023C1
:1031500084460E4D019267465F43E85D7E19A042AA
:1031600012D000280BD10A4B9C4662461B780833CC
:103170001370019B70707C557160B360FEBD0133AC
:103180000A2BE8D10320F9E70720F7E79867FF1F2C
:103190009467FF1F8020F8B5484BC0051B68C12409
:1031A0008360474BFF251A68012313434361454B56
:1031B000A4001A68444B40211A60444B1A68444BDF
:1031C0001A60444B1A59AA431A51C52292009E58BC
:1031D000AE433143802699509F583F49F6010F4036
:1031E0003E439E509E5880273602360A3043985000
:1031F00080201A5900020A4002431A5104341A5915
:10320000364E3F04324080263A431A511A59360648
:103210001202120A32431A5108341A5980260A40FF
:1032200002431A51C32292009F58B446AF4337431A
:103230009F509F58294E0F4007439F509F5837403B
:1032400080263604374380269F509F5836063F021B
:103250003F0A37439F50C0221F59AF433A431A5188
:103260001A591202120A1643C6221E5192009C5885
:10327000AC4365462C439C509C5800250C40204391
:103280009850C72080001A58154C1140C0221202D5
:103290000A431A50134B1B78DB08AB4201DC0020B9
:1032A000F8BD2378002B06D0A368002B00D09847E8
:1032B00001350C34EEE71220F2E7C046A443FF1FAD
:1032C000A043FF1FB0F000409067FF1FB4F0004024
:1032D0008C67FF1F00E100E0FF00FFFFFFFF00FF22
:1032E0009867FF1F9467FF1F030010B51F2809D8B8
:1032F000072200201340072404490A78A2431343FD
:103300000B7010BD00230620F5E7C0469467FF1F31
:10331000034A0449136800200B4013607047C046FD
:103320001CF00040FFFFC1FF054B06491B780A68EF
:1033300005485B0702401B0B134300200B607047DE
:103340009467FF1F1CF00040FFFFC1FF70B50C2504
:10335000FFF7EAFF0A4B1C780A4BE4086543ED18B7
:10336000002C01D1200070BD2B78002B06D06B689B
:10337000002B00D09847013C0C3DF1E71220F2E70A
:103380009467FF1F8C67FF1F1FB5002102220B00EF
:1033900001910091052000F0BFFD02230B490A684E
:1033A0001A42FCD120230393039B5A1E0392002B45
:1033B000FAD1074A1368002BFCDA0B246C44200076
:1033C000012100F031FC207804B010BD90C800400D
:1033D00000C8004013B504000A4B0193019B002B69
:1033E00001D1112016BDFFF7CFFF23000340044297
:1033F00005D0052000F038FD019B013BEDE71800EA
:10340000F0E7C046FFFFFF0707B500F005FC80228C
:103410000821D205936A0191002B01D107399162ED
:1034200002210C4A11600199481E01900029FAD12D
:1034300003311160053101910199481E0190002965
:10344000FAD11160002B02D18022D205936200F0E4
:1034500013FE07BD00C00040F0B52D4C89B02378A5
:10346000002B4FD1FEF7A8FA02232A4F03903A68A7
:103470001A42FCD120230693069B5A1E0692002B6B
:10348000FAD1254E3368002BFCDA0120FFF7A2FFAA
:10349000011E02D0112009B0F0BD030003220190EB
:1034A000009005AD9F2000F037FD0321280000F0BB
:1034B000BBFB02233A681A42FCD120230793079BE7
:1034C0005A1E0792002BFAD13368002BFCDA012038
:1034D000FFF780FF0028DDD10398FEF781FAAA7874
:1034E0006B7811041B020B4329780B4363601300B4
:1034F000113B0A49052B07D801239340A3600B60B9
:10350000012323700020C6E780231B03F6E7C04693
:103510008C43FF1F90C8004000C800409808FF1F60
:103520001E4B30B55A6818781D4B85B0D3185942D8
:103530004B4101210093002300F036FC194B1A4A3D
:1035400002259A6300221A6510325A658022C4212E
:103550009D65164B1648D202DA6789004258154B12
:1035600080241A4080231B041343435064234120CA
:103570000393E40500F006FA402000F003FA6562C8
:10358000039D6B1E0393002DFAD103236362FFF7A3
:103590003BFFA562FFF760FF05B030BD9843FF1FFA
:1035A00095FFFEF700C80040050001FF04E100E0C0
:1035B00000E100E0FFFF00FFF0B585B00700FEF777
:1035C000FBF9022305002D4C22681A42FCD120236E
:1035D0000093009B5A1E0092002BFAD1284E3368AC
:1035E000002BFCDA0120FFF7F5FE002803D01124A0
:1035F000200005B0F0BD234B2360022322681A424D
:10360000FCD120230193019B5A1E0192002BFAD179
:103610003368002BFCDA0120FFF7DCFE0028E6D13E
:10362000194B1F60022322681A42FCD12023029307
:10363000029B5A1E0292002BFAD13368002BFCDA4F
:103640000120FFF7C7FE0028D1D1104B23600223D1
:1036500022681A42FCD120230393039B5A1E039233
:10366000002BFAD13368002BFCDA0120FFF7B2FE01
:10367000041EBCD12800FEF7B3F9B9E790C800409A
:1036800000C8004001000006A8C8004001800001F9
:1036900010B50020FFF790FF10BD000010B5064BDD
:1036A00018705960FFF73CFF00211320034AFFF711
:1036B0004BFD002010BDC0469843FF1F2135FF1F62
:1036C000F0B5040085B003920291FEF775F98822E7
:1036D00063035B0B52051A438023DB059D6A80233D
:1036E000274F0092BA68002601901B039A420CD91A
:1036F000F82326001B041E401C4206D08022214BCA
:1037000052025E6219680A431A60002D0BD100F064
:1037100083FA02221C4B1A608023DB055A62013AAD
:103720009A6200F0A9FC0023039A934220D1002D55
:103730000AD100F071FA144B03221D608023DB05CF
:103740005A629D6200F098FC8023BA681B039A427B
:1037500008D9002E06D000220A4B0C495A621A687A
:103760000A401A600198FEF73BF9002005B0F0BD51
:10377000009A0299D2181278CA540133D4E7C0468D
:103780008C43FF1F00C8004000C00040FFFFFEFF49
:10379000F0B587B0029103920400FEF70DF9019095
:1037A00000F03AFA802302250122234EDB05356022
:1037B0005D629A6200F060FC204F3B682B42FCD1B6
:1037C00020230493049B5A1E0492002BFAD11C4D13
:1037D0002B68002BFCDA0120FFF7FCFD002802D04B
:1037E000112007B0F0BD2000039A029900F014FCEC
:1037F000022304003A681A42FCD120230593059B5A
:103800005A1E0592002BFAD12B68002BFCDA0120FE
:10381000FFF7E0FD051EE3D100F0FEF9802303224F
:10382000DB0535605A629D6200F026FC0198FEF7C8
:10383000D7F8E0B2D5E7C04600C0004090C80040CD
:1038400000C80040F0B5802489B00600FEF7B4F847
:10385000E405A36A02250393029000F0DDF9012339
:10386000304F3D606562A36200F006FC2E4C236879
:103870002B42FCD120230593059B5A1E0592002B59
:10388000FAD12A4D2B68002BFCDA0120FFF7A2FDAC
:10389000002803D01124200009B0F0BD244B236080
:1038A000022322681A42FCD120230693069B5A1E4B
:1038B0000692002BFAD12B68002BFCDA0120FFF7CF
:1038C00089FD021EE6D11B4B03211E6003000190FF
:1038D0000090202000F020FB022322681A42FCD135
:1038E00020230793079B5A1E0792002BFAD12B68BF
:1038F000002BFCDA0320FFF76DFD041ECAD100F097
:103900008BF980230322DB053C605A629C6200F045
:10391000B3FB039B002B01D1FFF776FD0298FEF766
:103920005FF8B8E700C0004090C8004000C8004001
:103930000100000694C8004007B50002019104226E
:10394000000A01A9FFF724FF0EBD000073B50500B2
:1039500005240B4AA3005B429B1819686B46DE1DC9
:103960003000FFF7A7FA022804D133782B55013C29
:10397000EFD276BD052CFCD00128FAD10230F8E751
:10398000140900111F2807D8012380228340D20583
:1039900091680B43936070473F2808D80123802229
:1039A00020388340D20551690B435361F3E75F2808
:1039B000F1D80123802240388340D205116A0B439D
:1039C0001362E8E71F2807D8012280218240C90539
:1039D0008B6893438B6070473F2808D80122802171
:1039E00020388240C9054B6993434B61F3E75F2858
:1039F000F1D80122802140388240C9050B6A9343E7
:103A00000B62E8E71F2810D880230200DB05153A77
:103A10001968012A06D820229143196019680A43BF
:103A20001A60704701228240F6E73F2811D88023B0
:103A30000200DB05353AD968032A06D810229143E3
:103A4000D960D9680A43DA60EBE701222038824066
:103A5000F5E75F28E5D842238022181A413B8340CE
:103A6000D205516A99435162516A0B435362D8E7B8
:103A700010B50400012813D1A022184992050B6843
:103A80005B015B0913430B60154B164A1968114023
:103A9000154A0A431A60402219680A431A6010BD89
:103AA0000028FCD101000A2000F0C6F821000B20FC
:103AB00000F0C2F8C0220A4B920019680A43402164
:103AC0001A601A688A431A60B022044912060B6809
:103AD0005B015B0913430B60E1E7C04614F0004053
:103AE0001CF000407F00FEFF80FD010072B6074A17
:103AF0001368013313600422054B1A600023054A42
:103B000013608022D2055360FEE7C0467808FF1F8D
:103B1000C0F00040C4F0004005490B68002B05D1FF
:103B2000044A0A6004490A60044A13607047C046A8
:103B3000140AFF1F841E0000380AFF1FC4F0004053
:103B40000023034A1360034A1360034A136070475B
:103B500054F0004040F1004044F1004002B471468E
:103B600049084900095649008E4402BC7047C046C6
:103B700002B4714649084900095C49008E4402BC00
:103B80007047C04603B47146490840004900095ACD
:103B900049008E4403BC704701B40248844601BC0E
:103BA000604700BF6DF6000001B40248844601BCC6
:103BB000604700BFBD5C010001B40248844601BCFF
:103BC000604700BFCD4C010001B40248844601BCEF
:103BD000604700BF090E000001B40248844601BCE2
:103BE000604700BFE927000001B40248844601BCD9
:103BF000604700BF0167010001B40248844601BC70
:103C0000604700BF8B52010001B40248844601BCEA
:103C1000604700BFF535010001B40248844601BC8D
:103C2000604700BF75A9000001B40248844601BC8A
:103C3000604700BF3D71010001B40248844601BCE9
:103C4000604700BF91A3001101B40248844601BC43
:103C5000604700BFCD0C010001B40248844601BC9E
:103C6000604700BF85C1000001B40248844601BC22
:103C7000604700BFC95C010001B40248844601BC32
:103C8000604700BF2144000001B40248844601BCE3
:103C9000604700BF6911010001B40248844601BCBD
:103CA000604700BFED6B010001B40248844601BCCF
:103CB000604700BF090E000001B40248844601BC01
:103CC000604700BF2D6C010001B40248844601BC6E
:103CD000604700BFD544010001B40248844601BCDE
:103CE000604700BF21A9000001B40248844601BC1E
:103CF000604700BFDD0A010001B40248844601BCF0
:103D0000604700BFC166010001B40248844601BC9F
:103D1000604700BFE512010001B40248844601BCBF
:103D2000604700BFF9ED000001B40248844601BCC1
:103D3000604700BFF90D010001B40248844601BC90
:103D4000604700BF8512010001B40248844601BCEF
:103D5000604700BFB352010001B40248844601BC71
:103D6000604700BFD9B0000001B40248844601BCDE
:103D7000604700BF116E000001B40248844601BCD8
:103D8000604700BF19FA000001B40248844601BC34
:103D9000604700BF7912010001B40248844601BCAB
:103DA000604700BF0D52010001B40248844601BCC7
:103DB000604700BFC56D010001B40248844601BCE4
:103DC000604700BFE9D4000001B40248844601BC4A
:103DD000604700BF71B0000001B40248844601BCD6
:103DE000604700BFADAE000001B40248844601BC8C
:103DF000604700BFD1AE000001B40248844601BC58
:103E0000604700BFE90B010001B40248844601BCD1
:103E1000604700BF6D0B010001B40248844601BC3D
:103E2000604700BFB70E000001B40248844601BCE1
:103E3000604700BFE917010001B40248844601BC95
:103E4000604700BFC115010001B40248844601BCAF
:103E5000604700BF9D6A000001B40248844601BC6F
:103E6000604700BF156B010001B40248844601BCE5
:103E7000604700BF0189000001B40248844601BCCC
:103E8000604700BFE94C010001B40248844601BC10
:103E9000604700BF51B8000001B40248844601BC2D
:103EA000604700BF01D7000001B40248844601BC4E
:103EB000604700BFF935010001B40248844601BCE7
:103EC000604700BF8552010001B40248844601BC2E
:103ED000604700BF0134010001B40248844601BCC0
:103EE000604700BFC9A9000001B40248844601BC74
:103EF000604700BFED68010001B40248844601BC80
:103F0000604700BF8944000001B40248844601BCF8
:103F1000604700BF8914010001B40248844601BC17
:103F2000604700BF496D010001B40248844601BCEE
:103F3000604700BFA9D8000001B40248844601BC14
:103F4000604700BF6137010001B40248844601BCEC
:103F5000604700BF4DF9000001B40248844601BC2F
:103F6000604700BFE9F6000001B40248844601BC86
:103F7000604700BF39B7001101B40248844601BC54
:103F8000604700BF53B9000001B40248844601BC39
:103F9000604700BFA1AF000001B40248844601BCE5
:103FA000604700BFC1A5000001B40248844601BCBF
:103FB000604700BFDD0C010001B40248844601BC2B
:103FC000604700BF016C010001B40248844601BC97
:103FD000604700BF0934010001B40248844601BCB7
:103FE000604700BF8937010001B40248844601BC24
:103FF000604700BFC1F7000001B40248844601BC1D
:10400000604700BF5976010001B40248844601BCF4
:10401000604700BFEDA5000001B40248844601BC22
:10402000604700BF9573010001B40248844601BC9B
:10403000604700BF75F8000001B40248844601BC27
:10404000604700BF8D11010001B40248844601BCE5
:10405000604700BF8D82000001B40248844601BC65
:10406000604700BFBD0B010001B40248844601BC9B
:10407000604700BF7997000001B40248844601BC44
:10408000604700BF9DA9000001B40248844601BCFE
:10409000604700BF0534010001B40248844601BCFA
:0840A000604700BFDD3F000096
:1040A800020000000AC000110100000000BE00115B
:1040B8000200000006C0001101000000E840FF1FD8
:1040C8000200000008BE0011010000002062FF1F6E
:1040D8000200000004C00011030000009461FF1FEB
:1040E80012000000020000000AC0001101000000D8
:1040F80048BE00110200000006C0001101000000C7
:1041080045BE00110200000052BE0011030000006D
:10411800CF61FF1F0200000004C00011030000006F
:10412800E461FF1F0200000006C00011010000004A
:1041380044BE00110200000050BE00110300000040
:10414800A561FF1F0200000004C000110300000069
:10415800C661FF1F020000000AC000110100000034
:1041680088BE00110200000006C000110100000016
:104178003142FF1F020000009ABE0011010000003A
:1041880083BE00110200000006C0001101000000FB
:104198003042FF1F0200000098BE0011010000001D
:1041A800EC61FF1F0200000006C0001101000000C2
:1041B8002F42FF1F0200000096BE00110100000000
:1041C80073BE00110200000006C0001101000000CB
:1041D8002E42FF1F0200000094BE001101000000E3
:1041E8006EBE00110200000006C0001101000000B0
:1041F8002D42FF1F0200000092BE001101000000C6
:1042080069BE00110200000006C000110100000094
:104218002C42FF1F0200000090BE001101000000A8
:1042280064BE001102020202020200000000000047
:1042380016150000CD4C0011934C0011F8BE00116A
:1042480090011D0018001800FFFF07010203040574
:104258000602010600000000000000000000000047
:104268000000000000000000000000000000000046
:1042780003000000020000000AC000110100000055
:1042880018BF00110200000006C000110100000064
:10429800EC42FF1F0200000022BF001101000000D5
:1042A8001A62FF1F0200000004C000110300000092
:1042B8008464FF1F0200000006C000110100000016
:1042C800EC42FF1F0200000020BF001101000000A7
:1042D8001C62FF1F0200000004C000110300000060
:1042E8007C64FF1F12A6A6A60000000000000000C4
:1042F800161500000001000000000111FFFF00007A
:104308005048593600000000000000000B0005006E
:10431800F0000000B4000028002800283075A00034
:10432800A000A000A00000080008E001F0001000B4
:104338001000100010001000100050005000500035
:1043480010001000D0070000000000000F0001005E
:104358000500307507001000010081FF0000000013
:10436800FF000000797500118173001111710011AF
:10437800FFFF0100FF000000959F0011119D001133
:10438800299C001100000000000000000000080047
:10439800040000003B0001085902E00188212800C0
:1043A800FF000000020000000AC000110100000028
:1043B800D0C000110200000006C00011010000007A
:1043C8002944FF1F0200000002C000110100000084
:1043D8005068FF1F0200000006C000110100000025
:1043E8002844FF1F0200000000C000110100000067
:1043F8002644FF1F0200000006C000110100000053
:104408002444FF1F02000000FEBF0011010000004D
:104418001C44FF1F180018001D0090010200000333
:1044280002020000020000000AC0001101000000A2
:10443800E4C000110200000006C0001101000000E5
:104448006C44FF1F02000000FCBF001100000000C8
:10445800000000000200000004C00011030000007A
:064468007068FF1F20FF39
:040000051FFF184180
:00000001FF
